:100000000C942A001895000018950000189500001F
:10001000189500001895000018950000189500002C
:10002000189500001895000018950000189500001C
:10003000189500001895000018950000189500000C
:1000400018950000189500001895000018950000FC
:10005000189500008FE58DBFC0E0E2E84E2E88E0E5
:100060008EBFD8E0F7E05F2EEEEFF7E0A0E6B0E05D
:1000700088278D933197E9F785E089B980E080BDC5
:1000800088E18AB966248CEF84BB0E94CC3586E077
:1000900086B98C9A8D9A8E9A8A9A8B9AD5988F98CF
:1000A000A098A198A6E4B1E0E8E3FAE70E946737D8
:1000B000979AA89AA99A80E0809368009498959856
:1000C000969805E515E525E53DE0A5E7B0E00D933B
:1000D0001D932D933C9305E515E525E531E0A9E752
:1000E000B0E00D931D932D933C9302E212E222E2C5
:1000F00030E0ADE7B0E00D931D932D933C9300ED00
:1001000019E623E030E0A1E8B0E00D931D932D93B4
:100110003C9301E617E520E030E0A5E8B0E00D9360
:100120001D932D933C93E4ECFCE50E94BF3381E0EA
:100130008093240100912401013318F011F00C94F4
:10014000BB000E94C233A4E2B1E0AD90BB24ADEF8E
:10015000B1E0AA0CBB1CAA0CBB1CAA0DBB1D0E94C3
:1001600074390E94BF33A4E2B1E08C918F5F8C930D
:1001700010F40C949A0081E08093F0010091F0015A
:100180000A3018F011F00C94CF000E94A321A0EFC8
:10019000B1E08C918F5F8C9310F40C94BE005A9256
:1001A0004A9284E190E0A42DB52D8D939C9382E03A
:1001B0000E94C9335A924A9283E0A42DB52D8C93A4
:1001C00081E00E94C9330E94142E249683E00E948D
:1001D000C5335A924A9284E190E0A42DB52D8D93B7
:1001E0009C9382E00E94C9335A924A9282E0A42DE5
:1001F000B52D8C9381E00E94C9330E94142E249661
:1002000083E00E94C5335A924A9284E190E0A42D83
:10021000B52D8D939C9382E00E94C9335A924A92E5
:1002200081E0A42DB52D8C9381E00E94C9330E94FA
:10023000142E249683E00E94C5330E94452E0E940E
:10024000BB1D5A924A9282E390E0A42DB52D8D9366
:100250009C9382E00E94C9335A924A9281E0A42D75
:10026000B52D8C9381E00E94C9330E94142E2496F0
:1002700083E00E94C533379A0E94A61E83E08093D4
:10028000650081E08093670081E08093EC0100913C
:10029000EC01033718F011F00C94600188E0ACEE2B
:1002A000B1E0AD90BB24A4E7B1E0AA0DBB1D8C93D7
:1002B000ACEEB1E08C918F5F8C9310F40C944701FD
:1002C00000E915E620E030E0A9E8B0E00D931D93C9
:1002D0002D933C938BE08093C300A8E1B1E0E8EC60
:1002E000F9E70E9474398091EF018F7D8093EF01CF
:1002F000ECEEFDE5A3ECB0E08C919927ADE8B0E021
:100300000E947F3987E08093C200E8E8FDE5A2EC17
:10031000B0E08C919927A1E9B0E00E947F39E4EB2D
:10032000FDE587E090E00E948639ADEBB0E00E94E9
:10033000673782B394E0892782BB0027A2E3B0E04D
:100340008C9183FB0EF401E041E0041711F00C9452
:10035000C10181E090E00E94C23482B394E0892719
:1003600082BB81E090E00E94C23482B394E089278E
:1003700082BB81E090E00E94C23482B394E089277E
:1003800082BB0E9435140E94FE14ADE8B0E00D91CE
:100390001D912D913C9142E050E060E070E00E94A0
:1003A0006534A5EAB0E04D935D936D937D93A9E824
:1003B000B0E00D911D912D913C91A5EAB0E04D91D9
:1003C0005D916D917C910E94323AA5E9B0E00D9368
:1003D0001D932D933D93ECECF9E70E944A39EDE82B
:1003E000F0E00E94E4370E9408380E945938EDE09E
:1003F000F0E0ADE9B0E00E94DA3A0027AFEEB1E0FC
:100400008C9185FB0EF401E040E0041711F00C9490
:100410001702A5E9B0E00D911D912D913C91A5EC3D
:10042000B0E00D931D932D933C930C942302A9E807
:10043000B0E00D911D912D913C91A5ECB0E00D9394
:100440001D932D933C93E5ECF0E00E94E4370E946D
:100450000838A1EAB0E00E94393883E790E0A5ECC3
:10046000B2E08D939C9300916700053011F00C94DD
:100470003B020C946E0981E08093F001A5ECB2E0A0
:100480004D915C91A0EFB1E00D9111270417150774
:1004900018F011F00C94D8060E94952C0091680079
:1004A000003011F40C945B020E94402580E08093A0
:1004B00068000C949901E5ECF0E0FA93EA930E944D
:1004C00001202296E0E7F0E0FA93EA930E94BE1F33
:1004D0002296EF93FF93E1E1F1E00E94B934FF919E
:1004E000EF9187E087B90E946D37A3EDB0E08D935F
:1004F0009C9386E087B90E946D37A5EDB0E08D939F
:100500009C930091F0010A3311F00C9410040E94A6
:10051000F021A1E3B1E0E8E6FAE70E9467375A92DA
:100520004A9289E1A42DB52D8C9381E00E94C933B4
:100530005A924A9280E0A42DB52D8C9381E00E94BE
:10054000C933E1E3F1E0FA93EA930E946A13269635
:1005500082E00E94C53300916700013011F00C94D5
:10056000C9025A924A9284E1A42DB52D8C9381E060
:100570000E94C9335A924A9280E0A42DB52D8C93E3
:1005800081E00E94C9330E94E90D249682E00E9416
:10059000C53300916700013081E009F080E08F935E
:1005A00000916700033081E009F080E09F91892B82
:1005B0008F9300916700043081E009F080E09F9103
:1005C000892B882311F40C942903009167000330D0
:1005D00011F00C94FB02E0EDF9E70E944A39E8EDD6
:1005E000F0E00E94E4370E94AF38EDE0F0E0A8EDC3
:1005F000B0E00E94DA3A5A924A9282E3A42DB52DD5
:100600008C9381E00E94C9335A924A9280E0A42DD3
:10061000B52D8C9381E00E94C9330E94540E24961C
:1006200082E00E94C53300916700033011F00C9402
:100630002903E0EDF9E70E944A39E8EDF0E00E9475
:10064000E4370E945938EDE0F0E0A8EDB0E00E94F8
:10065000DA3A00916700033081E009F080E08F937F
:100660000027AFEEB1E08C9185FB0EF401E040E095
:10067000041781E009F080E09F918923882311F419
:100680000C945A035A924A9285E5A42DB52D8C9369
:1006900081E00E94C9335A924A9280E0A42DB52D80
:1006A0008C9381E00E94C9330E947A12249682E0E2
:1006B0000E94C53300916700033081E009F080E0BB
:1006C0008F930027AFEEB1E08C9185FB0EF401E033
:1006D00040E0041781E009F080E09F91892388239E
:1006E00011F40C948B035A924A9289E1A42DB52DF2
:1006F0008C9381E00E94C9335A924A9280E0A42DE3
:10070000B52D8C9381E00E94C9330E94F512249686
:1007100082E00E94C53300916700013081E009F05A
:1007200080E08F9300916700023081E009F080E063
:100730009F91892B8F9300916700043081E009F02D
:1007400080E09F91892B882311F40C94BF035A9267
:100750004A9280E5A42DB52D8C9381E00E94C93387
:100760005A924A9280E0A42DB52D8C9381E00E948C
:10077000C9330E94D30E249682E00E94C5330091B3
:100780006700023081E009F080E08F930027AFEE30
:10079000B1E08C9185FB0EF401E040E0041781E0AC
:1007A00009F080E09F918923882311F40C94F003D1
:1007B0005A924A9289E1A42DB52D8C9381E00E9432
:1007C000C9335A924A9280E0A42DB52D8C9381E0D2
:1007D0000E94C9330E94DD11249682E00E94C53335
:1007E00000916700043011F00C940E045A924A9262
:1007F00084E1A42DB52D8C9381E00E94C9335A92D7
:100800004A9280E0A42DB52D8C9381E00E94C933DB
:100810000E942B11249682E00E94C5330C941C0484
:1008200000916700023011F00C941A040E94F0212C
:100830000C941C040E9443240091F00141E0041B2D
:10084000A2E2B1E00C93A2E2B1E08C91855F8C93BF
:1008500081E08093EC010091EC01013318F011F07C
:100860000C944A040091EC0147E0040FA4E2B1E0CB
:100870000C93A2E2B1E04C91A4E2B1E05C9190E073
:100880000E948936ACEEB1E08C918F5F8C9310F4AE
:100890000C942B0400916700013011F00C9480043B
:1008A00081E08093240100912401013318F011F0BC
:1008B0000C947E04E0E0F1E00E94E437E4E2F1E031
:1008C000A190BB24EDEFF1E0AA0CBB1CAA0CBB1C51
:1008D000EA0DFB1D0E94E9370E94533918F011F010
:1008E0000C9474040C9476040C946905A4E2B1E0B1
:1008F0008C918F5F8C9310F40C9453040C946905C5
:1009000000916700023011F00C94C904E4EDF9E79E
:100910000E944A39ECEFF0E00E94E4370E94AF38C1
:10092000EDE0F0E0ACE0B1E00E94DA3AE8EDF9E7A2
:100930000E944A39ECE0F1E00E94E4370E94593805
:10094000EDE0F0E0ACE0B1E00E94DA3AECE0F1E09A
:100950000E94E437E4EDF9E70E944A390E945339D6
:1009600018F011F00C94B6040C94BC04ACE0B1E0A7
:10097000ECEDF9E70E947439ECE0F1E00E94B83C3C
:10098000EDE0F0E00E94A637A4E2B1E0DC920C9426
:10099000690500916700033011F00C942205E4ED25
:1009A000F9E70E944A39E8EDF0E00E94E4370E943E
:1009B000AF38EDE0F0E0ACE0B1E00E94DA3AE0ED13
:1009C000F9E70E944A39ECE0F1E00E94E4370E9426
:1009D000AF38EDE0F0E0ACE0B1E00E94DA3AE0EEF2
:1009E000F9E70E944A39ECE0F1E00E94E4370E9406
:1009F0005938EDE0F0E0ACE0B1E00E94DA3AECE02A
:100A0000F1E00E94E437E4EDF9E70E944A390E94E0
:100A1000533918F011F00C940F050C941505ACE047
:100A2000B1E0ECEDF9E70E947439ECE0F1E00E94EE
:100A3000B83CEDE0F0E00E94A637A4E2B1E0DC9221
:100A40000C94690500916700043011F00C9469055D
:100A5000E4EDF9E70E944A39ECEDF0E00E94E4375A
:100A60000E94AF38EDE0F0E0ACE0B1E00E94DA3A8D
:100A7000E4EEF9E70E944A39ECE0F1E00E94E43745
:100A80000E945938EDE0F0E0ACE0B1E00E94DA3AC3
:100A9000ECE0F1E00E94E437E4EDF9E70E944A3926
:100AA0000E94533918F011F00C9458050C945E050F
:100AB000ACE0B1E0ECEDF9E70E947439ECE0F1E074
:100AC0000E94B83CEDE0F0E00E94A637A4E2B1E05D
:100AD000DC92A4E2B1E08C91895F8C938091240137
:100AE000A0EFB1E0AD90BB24A4E7B1E0AA0DBB1D1F
:100AF0008C93A2E2B1E04C91A0EFB1E0AD90BB24A9
:100B0000A4E7B1E0AA0DBB1D5C9191E00E9489367B
:100B10000091F001023018F011F00C9491050C9442
:100B2000A606A0EFB1E00D91112741E050E0041BB3
:100B3000150BAAEEB1E00D931C93AAEEB1E0AD90B7
:100B4000BC90A4E7B1E0AA0DBB1D0D911127A0EF49
:100B5000B1E0AD90BB24A4E7B1E0AA0DBB1D4D915F
:100B60005527041B150BA8EEB1E00D931C93A8EEBE
:100B7000B1E00D911C91003050E015071CF011F010
:100B80000C94C4050C94CB058091EF018068809390
:100B9000EF010C94D0058091EF018F778093EF01E6
:100BA000A8EEB1E08D919C910E940D34A8EEB1E0C9
:100BB0008D939C93A8EEB1E00D911C91003050E014
:100BC00015071CF011F00C94E7050C94A606A8EE8E
:100BD000B1E00D911C9142E050E00E94ED33AAEE8D
:100BE000B1E04D935C93A8EEB1E00D911C91AAEE9B
:100BF000B1E04D915C91041B150BA8EEB1E00D9393
:100C00001C938091EA018093EE01A0EFB1E00D9179
:100C1000112741E050E0041B150BAAEEB1E00D9343
:100C20001C93AAEEB1E0AD90BC90A4E7B1E0AA0D90
:100C3000BB1D8C918093ED01A2E2B1E08C918150BB
:100C40008C930091EE01003018F011F00C942A06FC
:100C50000C945F0681E08093EC014091EE010091DD
:100C6000EC01041718F011F00C945F060027AFEEAA
:100C7000B1E08C9187FB0EF401E041E0041711F024
:100C80000C944906ADEEB1E08C9181508C930C949C
:100C90004E06ADEEB1E08C918F5F8C93A2E2B1E095
:100CA0004C91ADEEB1E05C9191E00E948936ACEEE2
:100CB000B1E08C918F5F8C9310F40C942D06A2E21E
:100CC000B1E08C918F5F8C938091E8018093EE016D
:100CD0000091EE01003018F011F00C9471060C94A4
:100CE000A60681E08093EC014091EE010091EC01B9
:100CF000041718F011F00C94A6060027AFEEB1E02F
:100D00008C9187FB0EF401E041E0041711F00C9484
:100D10009006ADEEB1E08C9181508C930C949506C9
:100D2000ADEEB1E08C918F5F8C93A2E2B1E04C917B
:100D3000ADEEB1E05C9191E00E948936ACEEB1E09D
:100D40008C918F5F8C9310F40C9474060027AFEE97
:100D5000B1E08C9185FB0EF401E040E0041711F046
:100D60000C94D006EDE9F0E00E94E937E1EAF0E00A
:100D70000E94E4370E94EF38EDE0F0E0A1EAB0E035
:100D80000E94DA3AE1EAF0E00E94B83CEDE0F0E0DF
:100D90000E94A637A5ECB0E0EDE0FF270E94DA3A0A
:100DA000A0EFB1E08C918F5F8C9310F40C943E0215
:100DB000A9E6B0E00D911C91003050E015070CF051
:100DC00002C00C947207A9E6B0E00E94DC33A9E6E9
:100DD000B0E00D911C910A3050E0150711F00C9411
:100DE00072075A924A9280E590E0A42DB52D8D931A
:100DF0009C9382E00E94C9335A924A9282E0A42DC9
:100E0000B52D8C9381E00E94C9330E94142E249644
:100E100083E00E94C5335A924A9280E590E0A42D67
:100E2000B52D8D939C9382E00E94C9335A924A92C9
:100E300081E0A42DB52D8C9381E00E94C9330E94DE
:100E4000142E249683E00E94C53380E08A9380E0CC
:100E50008A9380E08A93E8EAF4E688278093640026
:100E60000E94B836E2E0F0E00E945C345A924A9266
:100E700080E590E0A42DB52D8D939C9382E00E9497
:100E8000C9335A924A9281E0A42DB52D8C9381E00A
:100E90000E94C9330E94142E249683E00E94C53319
:100EA0005A924A9280E590E0A42DB52D8D939C93A3
:100EB00082E00E94C9335A924A9282E0A42DB52D55
:100EC0008C9381E00E94C9330E94142E249683E003
:100ED0000E94C53380E090E0A9E6B0E08D939C933A
:100EE0000E942C360C9499015A924A9284E190E027
:100EF000A42DB52D8D939C9382E00E94C9335A9204
:100F00004A9281E0A42DB52D8C9381E00E94C933D3
:100F10000E94142E249683E00E94C5335A924A926E
:100F200084E190E0A42DB52D8D939C9382E00E94E6
:100F3000C9335A924A9282E0A42DB52D8C9381E058
:100F40000E94C9330E94142E249683E00E94C53368
:100F50005A924A9284E190E0A42DB52D8D939C93F2
:100F600082E00E94C9335A924A9284E0A42DB52DA2
:100F70008C9381E00E94C9330E94142E249683E052
:100F80000E94C53381E08093040380E080930303D3
:100F90000E94452E969895989498EF93FF93E1E1DF
:100FA000F1E00E94B934FF91EF9181E08093F0016C
:100FB0000091F0010A3018F011F00C94E9070E943A
:100FC000A321A0EFB1E08C918F5F8C9310F40C946F
:100FD000D80701EC16E12CE631E0ABECB2E00D9362
:100FE0001D932D933C938D9A8C9A9498ABECB2E020
:100FF00090E28D91983018F4392F992702C038E08B
:1010000098508795959808F4959A00000000949A56
:10101000EF93FF93E2E0F0E00E94B934FF91EF918B
:101020009498EF93FF93E2E0F0E00E94B934FF91CF
:10103000EF913A9531F79923E1F68D9A8C9A94982D
:10104000A4E0B3E098E08D91983018F4392F9927F7
:1010500002C038E098508795959808F4959A00005A
:101060000000949AEF93FF93E2E0F0E00E94B9341D
:10107000FF91EF919498EF93FF93E2E0F0E00E94EC
:10108000B934FF91EF913A9531F79923E1F6969AA9
:10109000000000000000000096980000000082B3ED
:1010A00094E0892782BB0E94243BAFEDB2E03FE091
:1010B0000E9436340E94213B41E050E060E070E045
:1010C000AFEDB2E00E94A33AA0E1B0E00D911D9116
:1010D0002D913C910E94373A11F00C94720893982C
:1010E0000C947308939A0E94243BAFECB2E03FE06B
:1010F0000E9436340E94213B0E94243BA9E0B3E0C9
:101100003FE00E9436340E94213B0E94243BA3EF23
:10111000B2E03FE00E9436340E94213B0000000014
:1011200000000000000000000000AFECB2E00E94F0
:10113000A33AABECB2E00D931D932D933D93A9E040
:10114000B3E00E94A33AA5E0B3E00D931D932D9365
:101150003D93A3EFB2E00E94A33AAFEEB2E00D934D
:101160001D932D933D9301E010E020E030E0A7ECCB
:10117000B2E00D931D932D933C93A5E0B3E04D9108
:101180005D916D917C91A7ECB2E00D911D912D9137
:101190003C910E94373A1CF011F00C946C09ABECB6
:1011A000B2E00D911D912D913C91AFEEB2E04D91C9
:1011B0005D916D917C910E942D3AABECB2E00D9364
:1011C0001D932D933D938D9A8C9A9498ABECB2E03D
:1011D00090E28D91983018F4392F992702C038E0A9
:1011E00098508795959808F4959A00000000949A75
:1011F000EF93FF93E2E0F0E00E94B934FF91EF91AA
:101200009498EF93FF93E2E0F0E00E94B934FF91ED
:10121000EF913A9531F79923E1F68D9A8C9A94984B
:10122000A4E0B3E098E08D91983018F4392F992715
:1012300002C038E098508795959808F4959A000078
:101240000000949AEF93FF93E2E0F0E00E94B9343B
:10125000FF91EF919498EF93FF93E2E0F0E00E940A
:10126000B934FF91EF913A9531F79923E1F6969AC7
:10127000000000000000000096980000EF93FF932C
:10128000E1E1F1E00E94B934FF91EF9187E087B985
:101290000E946D37A3EDB0E08D939C9386E087B9F3
:1012A0000E946D37A5EDB0E08D939C930000000087
:1012B000000032E0A3EDB0E00E94533400000000D3
:1012C000000032E0A5EDB0E00E945334A7ECB2E09C
:1012D0000E94CD330C94BD080C944F080E942C360C
:1012E000A1E3B1E0ECE7FAE70E9467375A924A922D
:1012F00080E0A42DB52D8C9381E00E94C9335A92D1
:101300004A9288E0A42DB52D8C9381E00E94C933C8
:10131000E1E3F1E0FA93EA930E946A13269682E0F1
:101320000E94C533A1E3B1E0E0E8FAE70E94673725
:101330005A924A9280E0A42DB52D8C9381E00E94B0
:10134000C9335A924A9280E1A42DB52D8C9381E045
:101350000E94C933E1E3F1E0FA93EA930E946A1331
:10136000269682E00E94C533A1E3B1E0E2E8FAE705
:101370000E9467375A924A9280E0A42DB52D8C9333
:1013800081E00E94C9335A924A9288E1A42DB52D7A
:101390008C9381E00E94C933E1E3F1E0FA93EA9390
:1013A0000E946A13269682E00E94C533A1E3B1E051
:1013B000E6E8FAE70E9467375A924A9280E0A42D45
:1013C000B52D8C9381E00E94C9335A924A9280E2F3
:1013D000A42DB52D8C9381E00E94C933E1E3F1E0A7
:1013E000FA93EA930E946A13269682E00E94C5331C
:1013F000A1E3B1E0EAE8FAE70E9467375A924A921D
:1014000080E0A42DB52D8C9381E00E94C9335A92BF
:101410004A9288E2A42DB52D8C9381E00E94C933B5
:10142000E1E3F1E0FA93EA930E946A13269682E0E0
:101430000E94C533A1E3B1E0EEE8FAE70E94673706
:101440005A924A9280E0A42DB52D8C9381E00E949F
:10145000C9335A924A9280E3A42DB52D8C9381E032
:101460000E94C933E1E3F1E0FA93EA930E946A1320
:10147000269682E00E94C533AAE6B7E0AF93BF93F9
:10148000E8E1F1E00E94E4370E94D73411E002E085
:10149000BF91AF910E94E539EAE6F7E0A6E2B1E03C
:1014A0000E94D53A5A924A9280E0A42DB52D8C9391
:1014B00081E00E94C9335A924A9288E3A42DB52D47
:1014C0008C9381E00E94C933E6E2F1E0FA93EA935B
:1014D0000E946A13269682E00E94C533ADE8B0E010
:1014E0000D911D912D913C9142E050E060E070E043
:1014F0000E946534A5EBB0E04D935D936D937D93B1
:10150000A9E8B0E00D911D912D913C91A5EBB0E0C3
:101510004D915D916D917C910E94323AA5ECB0E0C5
:101520000D931D932D933D93A1E3B1E0E5ECF0E025
:101530000E944D3AE1E3F1E0A6E2B1E01127222753
:1015400005E033E00E949A395A924A9288E1A42D2C
:10155000B52D8C9381E00E94C9335A924A9280E063
:10156000A42DB52D8C9381E00E94C933E6E2F1E011
:10157000FA93EA930E946A13269682E00E94C5338A
:10158000E5ECF0E0FA93EA930E9401202296E0E76E
:10159000F0E0FA93EA930E94BE1F22968AE090E060
:1015A0000E94C23487E087B90E946D37A3EDB0E096
:1015B0008D939C9386E087B90E946D37A5EDB0E0CE
:1015C0008D939C93EF93FF93E1E1F1E00E94B93496
:1015D000FF91EF910E94F0215A924A9288E1A42D46
:1015E000B52D8C9381E00E94C9335A924A9288E0CB
:1015F000A42DB52D8C9381E00E94C9330E94E90D82
:10160000249682E00E94C5335A924A9288E1A42D22
:10161000B52D8C9381E00E94C9335A924A9280E1A1
:10162000A42DB52D8C9381E00E94C9330E94D30E66
:10163000249682E00E94C5335A924A9288E1A42DF2
:10164000B52D8C9381E00E94C9335A924A9288E169
:10165000A42DB52D8C9381E00E94C9330E94540EB5
:10166000249682E00E94C5335A924A9288E1A42DC2
:10167000B52D8C9381E00E94C9335A924A9280E240
:10168000A42DB52D8C9381E00E94C9330E942B11AB
:10169000249682E00E94C5335A924A9288E1A42D92
:1016A000B52D8C9381E00E94C9335A924A9288E208
:1016B000A42DB52D8C9381E00E94C9330E949B0F0D
:1016C000249682E00E94C5335A924A9288E1A42D62
:1016D000B52D8C9381E00E94C9335A924A9280E3DF
:1016E000A42DB52D8C9381E00E94C9330E94631014
:1016F000249682E00E94C5335A924A9288E1A42D32
:10170000B52D8C9381E00E94C9335A924A9288E3A6
:10171000A42DB52D8C9381E00E94C9330E94F5124F
:10172000249682E00E94C533A9E8B0E00D911D9196
:101730002D913C91A5ECB0E00D931D932D933C931E
:10174000A1E3B1E0E5ECF0E00E944D3AE1E3F1E025
:10175000A6E2B1E01127222705E033E00E949A3982
:101760005A924A9289E3A42DB52D8C9381E00E9470
:10177000C9335A924A9280E0A42DB52D8C9381E012
:101780000E94C933E6E2F1E0FA93EA930E946A13F9
:10179000269682E00E94C533E5ECF0E0FA93EA93E6
:1017A0000E9401202296E0E7F0E0FA93EA930E947B
:1017B000BE1F22968AE090E00E94C23487E087B97B
:1017C0000E946D37A3EDB0E08D939C9386E087B9BE
:1017D0000E946D37A5EDB0E08D939C93EF93FF933E
:1017E000E1E1F1E00E94B934FF91EF910E94F02114
:1017F0005A924A9289E3A42DB52D8C9381E00E94E0
:10180000C9335A924A9288E0A42DB52D8C9381E079
:101810000E94C9330E94E90D249682E00E94C533DC
:101820005A924A9289E3A42DB52D8C9381E00E94AF
:10183000C9335A924A9280E1A42DB52D8C9381E050
:101840000E94C9330E94D30E249682E00E94C533C1
:101850005A924A9289E3A42DB52D8C9381E00E947F
:10186000C9335A924A9288E1A42DB52D8C9381E018
:101870000E94C9330E94540E249682E00E94C53310
:101880005A924A9289E3A42DB52D8C9381E00E944F
:10189000C9335A924A9280E2A42DB52D8C9381E0EF
:1018A0000E94C9330E942B11249682E00E94C53306
:1018B0005A924A9289E3A42DB52D8C9381E00E941F
:1018C000C9335A924A9288E2A42DB52D8C9381E0B7
:1018D0000E94C9330E949B0F249682E00E94C53368
:1018E0005A924A9289E3A42DB52D8C9381E00E94EF
:1018F000C9335A924A9280E3A42DB52D8C9381E08E
:101900000E94C9330E946310249682E00E94C5336E
:101910005A924A9289E3A42DB52D8C9381E00E94BE
:10192000C9335A924A9288E3A42DB52D8C9381E055
:101930000E94C9330E947A12249682E00E94C53325
:10194000ADE8B0E00D911D912D913C9142E050E049
:1019500060E070E00E946534A5EBB0E04D935D93CC
:101960006D937D93A9E8B0E00D911D912D913C916F
:10197000A5EBB0E04D915D916D917C910E942D3A67
:10198000A5ECB0E00D931D932D933D93A1E3B1E041
:10199000E5ECF0E00E944D3AE1E3F1E0A6E2B1E0CF
:1019A0001127222705E033E00E949A395A924A9281
:1019B0008AE5A42DB52D8C9381E00E94C9335A92FB
:1019C0004A9280E0A42DB52D8C9381E00E94C9330A
:1019D000E6E2F1E0FA93EA930E946A13269682E027
:1019E0000E94C533E5ECF0E0FA93EA930E940120EF
:1019F0002296E0E7F0E0FA93EA930E94BE1F229657
:101A00008AE090E00E94C23487E087B90E946D3777
:101A1000A3EDB0E08D939C9386E087B90E946D376B
:101A2000A5EDB0E08D939C93EF93FF93E1E1F1E09E
:101A30000E94B934FF91EF910E94F0215A924A928C
:101A40008AE5A42DB52D8C9381E00E94C9335A926A
:101A50004A9288E0A42DB52D8C9381E00E94C93371
:101A60000E94E90D249682E00E94C5335A924A9260
:101A70008AE5A42DB52D8C9381E00E94C9335A923A
:101A80004A9280E1A42DB52D8C9381E00E94C93348
:101A90000E94D30E249682E00E94C5335A924A9245
:101AA0008AE5A42DB52D8C9381E00E94C9335A920A
:101AB0004A9288E1A42DB52D8C9381E00E94C93310
:101AC0000E94540E249682E00E94C5335A924A9294
:101AD0008AE5A42DB52D8C9381E00E94C9335A92DA
:101AE0004A9280E2A42DB52D8C9381E00E94C933E7
:101AF0000E942B11249682E00E94C5335A924A928A
:101B00008AE5A42DB52D8C9381E00E94C9335A92A9
:101B10004A9288E2A42DB52D8C9381E00E94C933AE
:101B20000E949B0F249682E00E94C5335A924A92EB
:101B30008AE5A42DB52D8C9381E00E94C9335A9279
:101B40004A9280E3A42DB52D8C9381E00E94C93385
:101B50000E946310249682E00E94C5335A924A92F2
:101B60008AE5A42DB52D8C9381E00E94C9335A9249
:101B70004A9288E3A42DB52D8C9381E00E94C9334D
:101B80000E94DD11249682E00E94C5330E94952CAC
:101B900000916800003011F40C94D30D0E94402590
:101BA00080E08093680082B394E0892782BB0E9422
:101BB000031D89E190E00E94C23400916700053066
:101BC00011F40C9470090E942C360C949901F8942D
:101BD000FFCFE0E0F1E00E94E437E8EEF9E70E9491
:101BE0004A390E94533918F011F00C94F90D0C94F5
:101BF000010EA6E2B1E0E2E9FAE70E9467370C9431
:101C0000330EAAE6B7E0AF93BF93E0E0F1E00E94A5
:101C1000E4370E94D73411E002E0BF91AF910E94F7
:101C2000E539EAE6F7E0A6E2B1E00E94D53A8CE0B9
:101C30000E94D134E6E2F1E0A881B9810E94D53A50
:101C4000A6E2B1E0EAE9FAE70E946737E881F981A4
:101C5000A6E2B1E00E942D340E94D53A8CE0481AE9
:101C60008827580A22965A924A92AC81BD818C915B
:101C7000A42DB52D8C9381E00E94C9335A924A92CB
:101C8000AC81BD818C91A42DB52D8C9381E00E94F7
:101C9000C933E6E2F1E0FA93EA930E946A132696CA
:101CA00082E00E94C5330895AAE6B7E0AF93BF93E0
:101CB000E8EDF0E00E94E4370E94D73411E001E043
:101CC000BF91AF910E94E539EAE6F7E0A6E2B1E004
:101CD0000E94D53A8CE00E94D134E6E2F1E0A8817E
:101CE000B9810E94D53AA6E2B1E0EEE9FAE70E9496
:101CF0006737E881F981A6E2B1E00E942D340E94A5
:101D0000D53A8CE0481A8827580A2296E8EDF0E088
:101D10000E94E437ECEEF9E70E944A390E945339F9
:101D200018F011F00C94960E0C94B20E8CE00E94F8
:101D3000D134E6E2F1E0A881B9810E94D53AA6E269
:101D4000B1E0EEE9FAE70E946737E881F981A6E29F
:101D5000B1E00E942D340E94D53A8CE0481A8827C1
:101D6000580A22965A924A92AC81BD818C91A42D38
:101D7000B52D8C9381E00E94C9335A924A92AC816E
:101D8000BD818C91A42DB52D8C9381E00E94C93327
:101D9000E6E2F1E0FA93EA930E946A13269682E063
:101DA0000E94C5330895AAE6B7E0AF93BF93ECEF66
:101DB000F0E00E94E4370E94D73411E001E0BF91C7
:101DC000AF910E94E539EAE6F7E0A6E2B1E00E94B1
:101DD000D53AECEFF0E00E94E437E0EFF9E70E943B
:101DE0004A390E94533910F00C94120F8CE00E9473
:101DF000D134E6E2F1E0A881B9810E94D53AA6E2A9
:101E0000B1E0EEE9FAE70E946737E881F981A6E2DE
:101E1000B1E00E942D340E94D53A8CE0481A882700
:101E2000580A2296ECEFF0E00E94E437E4EFF9E77D
:101E30000E944A390E94533910F00C943B0F8CE0F9
:101E40000E94D134E6E2F1E0A881B9810E94D53A3E
:101E5000A6E2B1E0EEE9FAE70E946737E881F9818E
:101E6000A6E2B1E00E942D340E94D53A8CE0481AD7
:101E70008827580A2296ECEFF0E00E94E437E8EF5A
:101E8000F9E70E944A390E94533910F00C94640F0C
:101E90008CE00E94D134E6E2F1E0A881B9810E9491
:101EA000D53AA6E2B1E0EEE9FAE70E946737E881A9
:101EB000F981A6E2B1E00E942D340E94D53A8CE06F
:101EC000481A8827580A2296ECEFF0E00E94E4377F
:101ED000ECEFF9E70E944A390E94533918F011F0EB
:101EE0000C94740F0C947A0FA6E2B1E0E2E9FAE7E1
:101EF0000E9467375A924A92AC81BD818C91A42D81
:101F0000B52D8C9381E00E94C9335A924A92AC81DC
:101F1000BD818C91A42DB52D8C9381E00E94C93395
:101F2000E6E2F1E0FA93EA930E946A13269682E0D1
:101F30000E94C5330895AAE6B7E0AF93BF93E8EFD8
:101F4000F0E00E94E4370E94D73411E001E0BF9135
:101F5000AF910E94E539EAE6F7E0A6E2B1E00E941F
:101F6000D53AE8EFF0E00E94E437E0EFF9E70E94AD
:101F70004A390E94533910F00C94DA0F8CE00E9419
:101F8000D134E6E2F1E0A881B9810E94D53AA6E217
:101F9000B1E0EEE9FAE70E946737E881F981A6E24D
:101FA000B1E00E942D340E94D53A8CE0481A88276F
:101FB000580A2296E8EFF0E00E94E437E4EFF9E7F0
:101FC0000E944A390E94533910F00C9403108CE09F
:101FD0000E94D134E6E2F1E0A881B9810E94D53AAD
:101FE000A6E2B1E0EEE9FAE70E946737E881F981FD
:101FF000A6E2B1E00E942D340E94D53A8CE0481A46
:102000008827580A2296E8EFF0E00E94E437E8EFCC
:10201000F9E70E944A390E94533910F00C942C10B1
:102020008CE00E94D134E6E2F1E0A881B9810E94FF
:10203000D53AA6E2B1E0EEE9FAE70E946737E88117
:10204000F981A6E2B1E00E942D340E94D53A8CE0DD
:10205000481A8827580A2296E8EFF0E00E94E437F1
:10206000ECEFF9E70E944A390E94533918F011F059
:102070000C943C100C944210A6E2B1E0E2E9FAE7BD
:102080000E9467375A924A92AC81BD818C91A42DEF
:10209000B52D8C9381E00E94C9335A924A92AC814B
:1020A000BD818C91A42DB52D8C9381E00E94C93304
:1020B000E6E2F1E0FA93EA930E946A13269682E040
:1020C0000E94C5330895AAE6B7E0AF93BF93E4EF4B
:1020D000F0E00E94E4370E94D73411E001E0BF91A4
:1020E000AF910E94E539EAE6F7E0A6E2B1E00E948E
:1020F000D53AE4EFF0E00E94E437E0EFF9E70E9420
:102100004A390E94533910F00C94A2108CE00E94BE
:10211000D134E6E2F1E0A881B9810E94D53AA6E285
:10212000B1E0EEE9FAE70E946737E881F981A6E2BB
:10213000B1E00E942D340E94D53A8CE0481A8827DD
:10214000580A2296E4EFF0E00E94E437E4EFF9E762
:102150000E944A390E94533910F00C94CB108CE045
:102160000E94D134E6E2F1E0A881B9810E94D53A1B
:10217000A6E2B1E0EEE9FAE70E946737E881F9816B
:10218000A6E2B1E00E942D340E94D53A8CE0481AB4
:102190008827580A2296E4EFF0E00E94E437E8EF3F
:1021A000F9E70E944A390E94533910F00C94F41058
:1021B0008CE00E94D134E6E2F1E0A881B9810E946E
:1021C000D53AA6E2B1E0EEE9FAE70E946737E88186
:1021D000F981A6E2B1E00E942D340E94D53A8CE04C
:1021E000481A8827580A2296E4EFF0E00E94E43764
:1021F000ECEFF9E70E944A390E94533918F011F0C8
:102200000C9404110C940A11A6E2B1E0E2E9FAE799
:102210000E9467375A924A92AC81BD818C91A42D5D
:10222000B52D8C9381E00E94C9335A924A92AC81B9
:10223000BD818C91A42DB52D8C9381E00E94C93372
:10224000E6E2F1E0FA93EA930E946A13269682E0AE
:102250000E94C5330895AAE6B7E0AF93BF93ECEDB3
:10226000F0E00E94E4370E94D73411E001E0BF9112
:10227000AF910E94E539EAE6F7E0A6E2B1E00E94FC
:10228000D53AECEDF0E00E94E437E0EFF9E70E9488
:102290004A390E94533910F00C946A118CE00E9464
:1022A000D134E6E2F1E0A881B9810E94D53AA6E2F4
:1022B000B1E0EEE9FAE70E946737E881F981A6E22A
:1022C000B1E00E942D340E94D53A8CE0481A88274C
:1022D000580A2296ECEDF0E00E94E437E4EFF9E7CB
:1022E0000E944A390E94533910F00C9493118CE0EB
:1022F0000E94D134E6E2F1E0A881B9810E94D53A8A
:10230000A6E2B1E0EEE9FAE70E946737E881F981D9
:10231000A6E2B1E00E942D340E94D53A8CE0481A22
:102320008827580A2296ECEDF0E00E94E437E8EFA7
:10233000F9E70E944A390E94533910F00C94BC11FD
:102340008CE00E94D134E6E2F1E0A881B9810E94DC
:10235000D53AA6E2B1E0EEE9FAE70E946737E881F4
:10236000F981A6E2B1E00E942D340E94D53A8CE0BA
:10237000481A8827580A22965A924A92AC81BD81FF
:102380008C91A42DB52D8C9381E00E94C9335A9273
:102390004A92AC81BD818C91A42DB52D8C9381E0A6
:1023A0000E94C933E6E2F1E0FA93EA930E946A13CD
:1023B000269682E00E94C5330895EDE8F0E00E9481
:1023C000E4370E9408380E943E38E0E0FAE70E94B5
:1023D00041390E945938EDE0F0E0ACE0B1E00E94F4
:1023E000DA3AE4E0FAE70E944A39ECE0F1E00E94D0
:1023F000E4370E945938EDE0F0E0ACE0B1E00E9433
:10240000DA3AE8E1F1E00E94E937ECE0F1E00E941D
:10241000E4370E94AF38EDE0F0E0ACE0B1E00E94BC
:10242000DA3AAAE6B7E0AF93BF93ECE0F1E00E949E
:10243000E4370E94D73411E002E0BF91AF910E94CF
:10244000E539EAE6F7E0A6E2B1E00E94D53A8CE091
:102450000E94D134E6E2F1E0A881B9810E94D53A28
:10246000A6E2B1E0E0EAFAE70E946737E881F98185
:10247000A6E2B1E00E942D340E94D53A8CE0481AC1
:102480008827580A2296ECE0F1E00E94E437ECEF4E
:10249000F9E70E944A390E94533918F011F00C9460
:1024A00053120C945912A6E2B1E0E2EAFAE70E9454
:1024B00067375A924A92AC81BD818C91A42DB52D7B
:1024C0008C9381E00E94C9335A924A92AC81BD81BB
:1024D0008C91A42DB52D8C9381E00E94C933E6E246
:1024E000F1E0FA93EA930E946A13269682E00E9432
:1024F000C5330895EDE8F0E00E94E4370E94083803
:102500000E943E382F933F934F935F93E9E8F0E0AA
:102510000E94E4370E9408385F914F913F912F91BC
:102520000E945938EDE0F0E0ACE0B1E00E94DA3A08
:10253000ECE0F1E00E94273BEDE0F0E0ACE0B1E040
:102540000E94DA3AAAE6B7E0AF93BF93ECE0F1E07D
:102550000E94E4370E94D73411E000E0BF91AF91B0
:102560000E94E539EAE6F7E0A6E2B1E00E94D53A3A
:102570008CE00E94D134E6E2F1E0A881B9810E94AA
:10258000D53AA6E2B1E0EAEAFAE70E946737E881C5
:10259000F981A6E2B1E00E942D340E94D53A8CE088
:1025A000481A8827580A22965A924A92AC81BD81CD
:1025B0008C91A42DB52D8C9381E00E94C9335A9241
:1025C0004A92AC81BD818C91A42DB52D8C9381E074
:1025D0000E94C933E6E2F1E0FA93EA930E946A139B
:1025E000269682E00E94C5330895EDE8F0E00E944F
:1025F000E4370E940838ACE0B1E00E943938AAE61E
:10260000B7E0AF93BF93ECE0F1E00E94E4370E94A3
:10261000D73411E000E0BF91AF910E94E539EAE6BE
:10262000F7E0A6E2B1E00E94D53AECE0F1E00E94CA
:10263000E437E8E0FAE70E944A390E94533918F07B
:1026400011F00C9425130C942D13A6E2B1E0ECEAE2
:10265000FAE70E9467370C9449138CE00E94D1344A
:10266000E6E2F1E0A881B9810E94D53AA6E2B1E0A4
:10267000E4EBFAE70E946737E881F981A6E2B1E06E
:102680000E942D340E94D53A8CE0481A8827580AB7
:1026900022965A924A92AC81BD818C91A42DB52D7F
:1026A0008C9381E00E94C9335A924A92AC81BD81D9
:1026B0008C91A42DB52D8C9381E00E94C933E6E264
:1026C000F1E0FA93EA930E946A13269682E00E9450
:1026D000C533089581E00E94D13481E00E94D13455
:1026E00082E00E94D13481E00E94D13481E00E94D6
:1026F000D13481E00E94D13481E00E94D13481E064
:102700000E94D134A889B9890E941B3BAC85BD8544
:102710008C9381E0AE85BF858C93AC85BD854C9153
:10272000AE85BF850C91041718F011F00C942F148E
:10273000AE85BF858C91E889F98901E00A93AB8564
:10274000BC850E94E03AA6E4B1E0EA85FB85222739
:1027500091E00E947B37A885B9850C93A885B9853F
:102760000C91003011F00C94B91381E0A885B98563
:102770008C93A885B9858C9181508C93A885B98557
:102780000C9145E0049FAE81BF810C9280E0809364
:102790001C0100911C01043018F011F00C94271456
:1027A000ECE1FEE5AE81BF818C919927A885B985C2
:1027B0000E947C3980E1AA81BB818C9380E0809368
:1027C0001D0100911D01043018F011F00C94151436
:1027D000A885B9850C91AA81BB814C910423AC8159
:1027E000BD810C93AA89BB890C9140911D01040FF6
:1027F000A881B9810C93AC89BD894C91A881B9811C
:102800005C91AC81BD819C910E948936AA81BB817B
:102810000C9142E00E940B3B0C93ADE1B1E08C9136
:102820008F5F8C9310F40C94E113AC89BD898C916B
:102830008F5F8C93AE81BF818C918F5F8C93ACE165
:10284000B1E08C918F5F8C9310F40C94C913AE851A
:10285000BF858C918F5F8C9310F40C948D1389E05D
:10286000481A8827580A609608958AE08A9387E074
:102870008A938EE78A9387E08A938FEF8A930E94E8
:1028800008378EE78A9387E08A938EE78A9389E3F5
:102890008A938FEF8A930E9408378EE78A9389E3A1
:1028A0008A938AE08A9389E38A938FEF8A930E94BE
:1028B00008378AE08A9389E38A938AE08A9387E0DB
:1028C0008A938FEF8A930E94083700916700013046
:1028D00011F00C949C148FE78A9388E08A938FE719
:1028E0008A9388E38A9380E08A930E9408374FE7AF
:1028F00058E091E00E9489364FE756E191E00E944E
:1029000089364FE750E291E00E9489364FE755E261
:1029100091E00E9489364FE75AE291E00E948936A1
:102920004FE753E391E00E9489364FE758E391E087
:102930000E9489360C94CB148FE78A9388E08A939F
:102940008FE78A9388E38A9380E08A930E9408370E
:102950004FE758E091E00E9489364FE75FE091E051
:102960000E9489364FE757E191E00E9489364FE790
:102970005FE191E00E9489364FE758E291E00E94C2
:1029800089364FE750E391E00E9489364FE758E3DC
:1029900091E00E9489364BE05AE391E00E9489362B
:1029A00048E25AE391E00E94893644E45AE391E018
:1029B0000E94893641E65AE391E00E9489364DE74C
:1029C0005AE391E00E9489364BE056E091E00E9484
:1029D000893648E256E091E00E94893644E456E0A8
:1029E00091E00E94893641E656E091E00E948936E6
:1029F0004DE756E091E00E9489360895ADE8B0E0D9
:102A00000D911D912D913C9142E050E060E070E00D
:102A10000E946534A5EAB0E04D935D936D937D937C
:102A2000A9E8B0E00D911D912D913C91A5EAB0E08F
:102A30004D915D916D917C910E94323AA5E9B0E093
:102A40000D931D932D933D93ADE8B0E00D911D9135
:102A50002D913C9142E050E060E070E00E946534CE
:102A6000A9E9B0E04D935D936D937D930027AFEEA0
:102A7000B1E08C9185FB0EF401E040E0041711F009
:102A80000C946015A5E9B0E00D911D912D913C913C
:102A9000A5E9B0E00D931D932D933C93A1E3B1E024
:102AA000E5E9F0E00E944D3AE1E3F1E0A6E2B1E0B1
:102AB0001127222705E033E00E949A390C9466150D
:102AC000A6E2B1E0E6EBFAE70E9467375A924A9233
:102AD00080E0A42DB52D8C9381E00E94C9335A92D9
:102AE0004A928BE3A42DB52D8C9381E00E94C933CB
:102AF000E6E2F1E0FA93EA930E946A13269682E0F6
:102B00000E94C5330027AFEEB1E08C9185FB0EF437
:102B100001E040E0041711F00C94A415A5E9B0E021
:102B20000D911D912D913C91A9E9B0E04D915D91E0
:102B30006D917C910E942D3AA5E9B0E00D931D9313
:102B40002D933D930C94B015A9E8B0E00D911D9123
:102B50002D913C91A5E9B0E00D931D932D933C93ED
:102B6000A1E3B1E0E5E9F0E00E944D3AE1E3F1E0F4
:102B7000A6E2B1E01127222705E033E00E949A394E
:102B80005A924A9288E3A42DB52D8C9381E00E943D
:102B9000C9335A924A928BE3A42DB52D8C9381E0D0
:102BA0000E94C933E6E2F1E0FA93EA930E946A13C5
:102BB000269682E00E94C5330027AFEEB1E08C91EB
:102BC00085FB0EF401E040E0041711F00C940E16A2
:102BD000A5E9B0E00D911D912D913C91A9E9B0E0DE
:102BE0004D915D916D917C910E942D3AA5E9B0E0E7
:102BF0000D931D932D933D93A1E3B1E0E5E9F0E042
:102C00000E944D3AE1E3F1E0A6E2B1E0112722276C
:102C100005E033E00E949A390C941416A6E2B1E064
:102C2000EEEBFAE70E9467375A924A9281E6A42DAA
:102C3000B52D8C9381E00E94C9335A924A928BE35E
:102C4000A42DB52D8C9381E00E94C933E6E2F1E01A
:102C5000FA93EA930E946A13269682E00E94C53393
:102C600000916700013011F00C94D017A1E3B1E09E
:102C7000EAE9FAE70E9467375A924A9280E0A42D67
:102C8000B52D8C9381E00E94C9335A924A928DE00F
:102C9000A42DB52D8C9381E00E94C933E1E3F1E0CE
:102CA000FA93EA930E946A13269682E00E94C53343
:102CB000A1E3B1E0EAE9FAE70E9467375A924A9243
:102CC00080E0A42DB52D8C9381E00E94C9335A92E7
:102CD0004A9285E1A42DB52D8C9381E00E94C933E1
:102CE000E1E3F1E0FA93EA930E946A13269682E008
:102CF0000E94C533A1E3B1E0EAE9FAE70E94673731
:102D00005A924A9280E0A42DB52D8C9381E00E94C6
:102D1000C9335A924A928DE1A42DB52D8C9381E04E
:102D20000E94C933E1E3F1E0FA93EA930E946A1347
:102D3000269682E00E94C533A1E3B1E0EAE9FAE712
:102D40000E9467375A924A9280E0A42DB52D8C9349
:102D500081E00E94C9335A924A9286E2A42DB52D91
:102D60008C9381E00E94C933E1E3F1E0FA93EA93A6
:102D70000E946A13269682E00E94C533A1E3B1E067
:102D8000EAE9FAE70E9467375A924A9280E0A42D56
:102D9000B52D8C9381E00E94C9335A924A928EE2FB
:102DA000A42DB52D8C9381E00E94C933E1E3F1E0BD
:102DB000FA93EA930E946A13269682E00E94C53332
:102DC000A1E3B1E0E6ECFAE70E9467375A924A9233
:102DD00080E0A42DB52D8C9381E00E94C9335A92D6
:102DE0004A9286E0A42DB52D8C9381E00E94C933D0
:102DF000E1E3F1E0FA93EA930E946A13269682E0F7
:102E00000E94C533A1E3B1E0EAECFAE70E9467371C
:102E10005A924A9280E0A42DB52D8C9381E00E94B5
:102E2000C9335A924A9284E1A42DB52D8C9381E046
:102E30000E94C933E1E3F1E0FA93EA930E946A1336
:102E4000269682E00E94C533A1E3B1E0ECECFAE7FC
:102E50000E9467375A924A9280E0A42DB52D8C9338
:102E600081E00E94C9335A924A928EE1A42DB52D79
:102E70008C9381E00E94C933E1E3F1E0FA93EA9395
:102E80000E946A13269682E00E94C533A1E3B1E056
:102E9000EEECFAE70E9467375A924A9280E0A42D3E
:102EA000B52D8C9381E00E94C9335A924A9285E3F2
:102EB000A42DB52D8C9381E00E94C933E1E3F1E0AC
:102EC000FA93EA930E946A13269682E00E94C53321
:102ED000A1E3B1E0E2EDFAE70E9467375A924A9225
:102EE00083E0A42DB52D8C9381E00E94C9335A92C2
:102EF0004A9283E2A42DB52D8C9381E00E94C933C0
:102F0000E1E3F1E0FA93EA930E946A13269682E0E5
:102F10000E94C533A1E3B1E0E4EDFAE70E94673710
:102F20005A924A9283E0A42DB52D8C9381E00E94A1
:102F3000C9335A924A9288E2A42DB52D8C9381E030
:102F40000E94C933E1E3F1E0FA93EA930E946A1325
:102F5000269682E00E94C533A1E3B1E0E6EDFAE7F0
:102F60000E9467375A924A9283E0A42DB52D8C9324
:102F700081E00E94C9335A924A9281E3A42DB52D73
:102F80008C9381E00E94C933E1E3F1E0FA93EA9384
:102F90000E946A13269682E00E94C5330C94AE1CF0
:102FA00000916700023011F00C947019A1E3B1E0B8
:102FB000EEE9FAE70E9467375A924A9280E0A42D20
:102FC000B52D8C9381E00E94C9335A924A9284E1D4
:102FD000A42DB52D8C9381E00E94C933E1E3F1E08B
:102FE000FA93EA930E946A13269682E00E94C53300
:102FF000A1E3B1E0EEE9FAE70E9467375A924A92FC
:1030000080E0A42DB52D8C9381E00E94C9335A92A3
:103010004A928EE1A42DB52D8C9381E00E94C93394
:10302000E1E3F1E0FA93EA930E946A13269682E0C4
:103030000E94C533A1E3B1E0EEE9FAE70E946737E9
:103040005A924A9283E0A42DB52D8C9381E00E9480
:10305000C9335A924A9283E2A42DB52D8C9381E014
:103060000E94C933E1E3F1E0FA93EA930E946A1304
:10307000269682E00E94C533A1E3B1E0EEE9FAE7CB
:103080000E9467375A924A9283E0A42DB52D8C9303
:1030900081E00E94C9335A924A9288E2A42DB52D4C
:1030A0008C9381E00E94C933E1E3F1E0FA93EA9363
:1030B0000E946A13269682E00E94C533A1E3B1E024
:1030C000EEE9FAE70E9467375A924A9283E0A42D0C
:1030D000B52D8C9381E00E94C9335A924A9281E3C4
:1030E000A42DB52D8C9381E00E94C933E1E3F1E07A
:1030F000FA93EA930E946A13269682E00E94C533EF
:10310000A1E3B1E0E8EDFAE70E9467375A924A92EC
:1031100080E0A42DB52D8C9381E00E94C9335A9292
:103120004A9286E0A42DB52D8C9381E00E94C9338C
:10313000E1E3F1E0FA93EA930E946A13269682E0B3
:103140000E94C533A1E3B1E0ECEDFAE70E946737D6
:103150005A924A9280E0A42DB52D8C9381E00E9472
:10316000C9335A924A928DE0A42DB52D8C9381E0FB
:103170000E94C933E1E3F1E0FA93EA930E946A13F3
:10318000269682E00E94C533A1E3B1E0E0EEFAE7C3
:103190000E9467375A924A9280E0A42DB52D8C93F5
:1031A00081E00E94C9335A924A9285E1A42DB52D3F
:1031B0008C9381E00E94C933E1E3F1E0FA93EA9352
:1031C0000E946A13269682E00E94C533A1E3B1E013
:1031D000E4EEFAE70E9467375A924A9280E0A42D03
:1031E000B52D8C9381E00E94C9335A924A928DE1A9
:1031F000A42DB52D8C9381E00E94C933E1E3F1E069
:10320000FA93EA930E946A13269682E00E94C533DD
:10321000A1E3B1E0E8EEFAE70E9467375A924A92DA
:1032200080E0A42DB52D8C9381E00E94C9335A9281
:103230004A9286E2A42DB52D8C9381E00E94C93379
:10324000E1E3F1E0FA93EA930E946A13269682E0A2
:103250000E94C533A1E3B1E0ECEEFAE70E946737C4
:103260005A924A9280E0A42DB52D8C9381E00E9461
:10327000C9335A924A928EE2A42DB52D8C9381E0E7
:103280000E94C933E1E3F1E0FA93EA930E946A13E2
:10329000269682E00E94C533A1E3B1E0E0EFFAE7B1
:1032A0000E9467375A924A9280E0A42DB52D8C93E4
:1032B00081E00E94C9335A924A9285E3A42DB52D2C
:1032C0008C9381E00E94C933E1E3F1E0FA93EA9341
:1032D0000E946A13269682E00E94C5330C94AE1CAD
:1032E00000916700033011F00C94101BA1E3B1E0D2
:1032F000EEE9FAE70E9467375A924A9280E0A42DDD
:10330000B52D8C9381E00E94C9335A924A9284E190
:10331000A42DB52D8C9381E00E94C933E1E3F1E047
:10332000FA93EA930E946A13269682E00E94C533BC
:10333000A1E3B1E0EEE9FAE70E9467375A924A92B8
:1033400080E0A42DB52D8C9381E00E94C9335A9260
:103350004A928EE1A42DB52D8C9381E00E94C93351
:10336000E1E3F1E0FA93EA930E946A13269682E081
:103370000E94C533A1E3B1E0EEE9FAE70E946737A6
:103380005A924A9283E0A42DB52D8C9381E00E943D
:10339000C9335A924A9283E2A42DB52D8C9381E0D1
:1033A0000E94C933E1E3F1E0FA93EA930E946A13C1
:1033B000269682E00E94C533A1E3B1E0EEE9FAE788
:1033C0000E9467375A924A9283E0A42DB52D8C93C0
:1033D00081E00E94C9335A924A9288E2A42DB52D09
:1033E0008C9381E00E94C933E1E3F1E0FA93EA9320
:1033F0000E946A13269682E00E94C533A1E3B1E0E1
:10340000EEE9FAE70E9467375A924A9283E0A42DC8
:10341000B52D8C9381E00E94C9335A924A9281E380
:10342000A42DB52D8C9381E00E94C933E1E3F1E036
:10343000FA93EA930E946A13269682E00E94C533AB
:10344000A1E3B1E0E4EFFAE70E9467375A924A92AB
:1034500080E0A42DB52D8C9381E00E94C9335A924F
:103460004A9286E0A42DB52D8C9381E00E94C93349
:10347000E1E3F1E0FA93EA930E946A13269682E070
:103480000E94C533A1E3B1E0E0EEFAE70E9467379E
:103490005A924A9280E0A42DB52D8C9381E00E942F
:1034A000C9335A924A928DE0A42DB52D8C9381E0B8
:1034B0000E94C933E1E3F1E0FA93EA930E946A13B0
:1034C000269682E00E94C533A1E3B1E0E8EEFAE778
:1034D0000E9467375A924A9280E0A42DB52D8C93B2
:1034E00081E00E94C9335A924A9285E1A42DB52DFC
:1034F0008C9381E00E94C933E1E3F1E0FA93EA930F
:103500000E946A13269682E00E94C533A1E3B1E0CF
:10351000E0EFFAE70E9467375A924A9280E0A42DC2
:10352000B52D8C9381E00E94C9335A924A928DE165
:10353000A42DB52D8C9381E00E94C933E1E3F1E025
:10354000FA93EA930E946A13269682E00E94C5339A
:10355000A1E3B1E0E8EFFAE70E9467375A924A9296
:1035600080E0A42DB52D8C9381E00E94C9335A923E
:103570004A9286E2A42DB52D8C9381E00E94C93336
:10358000E1E3F1E0FA93EA930E946A13269682E05F
:103590000E94C533A1E3B1E0ECEFFAE70E94673780
:1035A0005A924A9280E0A42DB52D8C9381E00E941E
:1035B000C9335A924A928EE2A42DB52D8C9381E0A4
:1035C0000E94C933E1E3F1E0FA93EA930E946A139F
:1035D000269682E00E94C533A1E3B1E0E0E0FBE77C
:1035E0000E9467375A924A9280E0A42DB52D8C93A1
:1035F00081E00E94C9335A924A9285E3A42DB52DE9
:103600008C9381E00E94C933E1E3F1E0FA93EA93FD
:103610000E946A13269682E00E94C5330C94AE1C69
:1036200000916700043011F00C94AE1CA1E3B1E0EE
:10363000EEE9FAE70E9467375A924A9280E0A42D99
:10364000B52D8C9381E00E94C9335A924A9284E14D
:10365000A42DB52D8C9381E00E94C933E1E3F1E004
:10366000FA93EA930E946A13269682E00E94C53379
:10367000A1E3B1E0EEE9FAE70E9467375A924A9275
:1036800080E0A42DB52D8C9381E00E94C9335A921D
:103690004A928EE1A42DB52D8C9381E00E94C9330E
:1036A000E1E3F1E0FA93EA930E946A13269682E03E
:1036B0000E94C533A1E3B1E0EEE9FAE70E94673763
:1036C0005A924A9283E0A42DB52D8C9381E00E94FA
:1036D000C9335A924A9283E2A42DB52D8C9381E08E
:1036E0000E94C933E1E3F1E0FA93EA930E946A137E
:1036F000269682E00E94C533A1E3B1E0EEE9FAE745
:103700000E9467375A924A9283E0A42DB52D8C937C
:1037100081E00E94C9335A924A9288E2A42DB52DC5
:103720008C9381E00E94C933E1E3F1E0FA93EA93DC
:103730000E946A13269682E00E94C533A1E3B1E09D
:10374000EEE9FAE70E9467375A924A9283E0A42D85
:10375000B52D8C9381E00E94C9335A924A9281E33D
:10376000A42DB52D8C9381E00E94C933E1E3F1E0F3
:10377000FA93EA930E946A13269682E00E94C53368
:10378000A1E3B1E0E8EDFAE70E9467375A924A9266
:1037900080E0A42DB52D8C9381E00E94C9335A920C
:1037A0004A9286E0A42DB52D8C9381E00E94C93306
:1037B000E1E3F1E0FA93EA930E946A13269682E02D
:1037C0000E94C533A1E3B1E0E4E0FBE70E94673764
:1037D0005A924A9280E0A42DB52D8C9381E00E94EC
:1037E000C9335A924A928DE0A42DB52D8C9381E075
:1037F0000E94C933E1E3F1E0FA93EA930E946A136D
:10380000269682E00E94C533A1E3B1E0E8E0FBE741
:103810000E9467375A924A9280E0A42DB52D8C936E
:1038200081E00E94C9335A924A9285E1A42DB52DB8
:103830008C9381E00E94C933E1E3F1E0FA93EA93CB
:103840000E946A13269682E00E94C533A1E3B1E08C
:10385000ECE0FBE70E9467375A924A9280E0A42D81
:10386000B52D8C9381E00E94C9335A924A928DE122
:10387000A42DB52D8C9381E00E94C933E1E3F1E0E2
:10388000FA93EA930E946A13269682E00E94C53357
:10389000A1E3B1E0E0E1FBE70E9467375A924A9268
:1038A00080E0A42DB52D8C9381E00E94C9335A92FB
:1038B0004A9286E2A42DB52D8C9381E00E94C933F3
:1038C000E1E3F1E0FA93EA930E946A13269682E01C
:1038D0000E94C533A1E3B1E0E4EEFAE70E94673746
:1038E0005A924A9280E0A42DB52D8C9381E00E94DB
:1038F000C9335A924A928EE2A42DB52D8C9381E061
:103900000E94C933E1E3F1E0FA93EA930E946A135B
:10391000269682E00E94C533A1E3B1E0E4E1FBE733
:103920000E9467375A924A9280E0A42DB52D8C935D
:1039300081E00E94C9335A924A9285E3A42DB52DA5
:103940008C9381E00E94C933E1E3F1E0FA93EA93BA
:103950000E946A13269682E00E94C5330E94031DCE
:1039600000916700013011F00C94BE1CA1E3B1E09E
:10397000E8E1FBE70E9467370C94E61C00916700C2
:10398000023011F00C94CC1CA1E3B1E0ECE1FBE7B8
:103990000E9467370C94E61C00916700033011F019
:1039A0000C94DA1CA1E3B1E0E0E2FBE70E94673788
:1039B0000C94E61C00916700043011F00C94E61C96
:1039C000A1E3B1E0E4E2FBE70E9467375A924A9232
:1039D00083E2A42DB52D8C9381E00E94C9335A92C5
:1039E0004A928BE3A42DB52D8C9381E00E94C933BC
:1039F000E1E3F1E0FA93EA930E946A13269682E0EB
:103A00000E94C5330895EDEBF0E0A1E3B1E00E9420
:103A1000D53A5A924A9280E0A42DB52D8C9381E03C
:103A20000E94C9335A924A9280E0A42DB52D8C93FE
:103A300081E00E94C933E1E3F1E0FA93EA930E9446
:103A40006A13269682E00E94C5330027A3E3B0E004
:103A50008C9181FB0EF401E041E0041781E009F054
:103A600080E08F930027A3E3B0E08C9180FB0EF4FD
:103A700001E041E0041781E009F080E09F91892B8B
:103A8000882311F40C94AA1D00916500013011F0F7
:103A90000C94521DA1E3B1E0E8E2FBE70E94673716
:103AA0000C948E1D023011F00C946C1D0091670077
:103AB000053011F00C94641DA1E3B1E0EAE2FBE7EC
:103AC0000E9467370C946A1DA1E3B1E0ECE2FBE7CA
:103AD0000E9467370C948E1D033011F00C94781DF2
:103AE000A1E3B1E0E0E8FAE70E9467370C948E1D8D
:103AF000043011F00C94841DA1E3B1E0EEE2FBE789
:103B00000E9467370C948E1D053011F00C948E1DA9
:103B1000A1E3B1E0E0E3FBE70E9467375A924A92E3
:103B200088E7A42DB52D8C9381E00E94C9335A9269
:103B30004A9280E0A42DB52D8C9381E00E94C93378
:103B4000E1E3F1E0FA93EA930E946A13269682E099
:103B50000E94C5330027A0E3B0E08C9187FB0EF4F0
:103B600001E040E0041711F00C94BA1D8CE291E0E2
:103B70000E94C23408950E942C3684E190E00E9495
:103B8000C2345A924A928AE090E0A42DB52D8D93CA
:103B90009C9382E00E94C9335A924A9283E0A42DFA
:103BA000B52D8C9381E00E94C9330E94142E249677
:103BB00083E00E94C53380E08A9380E08A9380E0AE
:103BC0008A93E8EAF4E68827809364000E94B83676
:103BD000E1E0F0E00E945C340E942C3684E190E049
:103BE0000E94C2345A924A9284E190E0A42DB52DED
:103BF0008D939C9382E00E94C9335A924A9283E04B
:103C0000A42DB52D8C9381E00E94C9330E94142EFF
:103C1000249683E00E94C53380E08A9380E08A93F3
:103C200080E08A93E8E0FFE58827809364000E94A3
:103C3000B836E2E0F0E00E945C340E942C365A92E2
:103C40004A928AE090E0A42DB52D8D939C9382E05A
:103C50000E94C9335A924A9283E0A42DB52D8C93C9
:103C600081E00E94C9330E94142E249683E00E94B2
:103C7000C533A1E3B1E0E2E3FBE70E9467375A9264
:103C80004A928DE1A42DB52D8C9381E00E94C93319
:103C90005A924A9284E1A42DB52D8C9381E00E9422
:103CA000C933E1E3F1E0FA93EA930E946A1326969E
:103CB00082E00E94C533A1E3B1E0E2E4FBE70E94A9
:103CC00067375A924A9289E1A42DB52D8C9381E0F1
:103CD0000E94C9335A924A928EE1A42DB52D8C933D
:103CE00081E00E94C933E1E3F1E0FA93EA930E9494
:103CF0006A13269682E00E94C533A1E3B1E0E4E5B1
:103D0000FBE70E9467375A924A928EE1A42DB52DA7
:103D10008C9381E00E94C9335A924A9282E3A42D87
:103D2000B52D8C9381E00E94C933E1E3F1E0FA9371
:103D3000EA930E946A13269682E00E94C533E1E06E
:103D4000F0E00E945C340E942C3608950E942C36CC
:103D500084E690E00E94C234A1E3B1E0E6E6FBE72E
:103D60000E9467375A924A928AE5A42DB52D8C930A
:103D700081E00E94C9335A924A9281E0A42DB52D68
:103D80008C9381E00E94C933E1E3F1E0FA93EA9376
:103D90000E946A13269682E00E94C533A1E3B1E037
:103DA000EAE6FBE70E9467375A924A9289E1A42D1E
:103DB000B52D8C9381E00E94C9335A924A9284E1D6
:103DC000A42DB52D8C9381E00E94C933E1E3F1E08D
:103DD000FA93EA930E946A13269682E00E94C53302
:103DE000A1E3B1E0E8E7FBE70E9467375A924A9205
:103DF00089E1A42DB52D8C9381E00E94C9335A929C
:103E00004A928EE1A42DB52D8C9381E00E94C93396
:103E1000E1E3F1E0FA93EA930E946A13269682E0C6
:103E20000E94C533A1E3B1E0ECE8FBE70E946737ED
:103E30005A924A9289E1A42DB52D8C9381E00E947B
:103E4000C9335A924A9282E3A42DB52D8C9381E016
:103E50000E94C933E1E3F1E0FA93EA930E946A1306
:103E6000269682E00E94C53384E690E0A9E6B0E0A1
:103E70008D939C9380E080936800A9E6B0E00E9457
:103E8000E33382B394E0892782BBA1E3B1E0E9E6A2
:103E9000F0E00E94523AE1E3F1E0A6E2B1E011273E
:103EA000222702E030E00E949A395A924A928CE32B
:103EB000A42DB52D8C9381E00E94C9335A924A9269
:103EC0008AE0A42DB52D8C9381E00E94C933E6E2EF
:103ED000F1E0FA93EA930E946A13269682E00E9428
:103EE000C5338AE090E00E94C2340E94952C0027DE
:103EF000A9E3B0E08C9185FB0EF401E041E00417EA
:103F000011F00C94861F81E0809368000091680096
:103F1000013011F00C949D1F0E942C3680E08A9392
:103F200080E08A9380E08A93E4E4F2E68827809335
:103F300064000E94B8360C94740700916800013048
:103F400018F011F00C94A61F0C94AE1F0E942C3692
:103F500080E090E0A9E6B0E08D939C93A9E6B0E004
:103F60000D911C91003050E0150711F00C943D1F8D
:103F700080E0809368000E942C3608958D9A8C9A78
:103F80009498A881B98190E28D91983018F4392FD6
:103F9000992702C038E098508795959808F4959A2B
:103FA00000000000949A00000000949800000000B7
:103FB0003A9591F7992341F781E0809374008D9AA7
:103FC0008C9A9498A4E7B0E098E08D91983018F41A
:103FD000392F992702C038E098508795959808F4B2
:103FE000959A00000000949A000000009498000048
:103FF00000003A9591F7992341F7969A0000969818
:104000000895A881B9810D911D912D913C91A9EC44
:10401000B0E00D931D932D933C9380E197E2A1EDC9
:10402000B0E08D939C9300E010E020E030E0A0E74A
:10403000B0E00D931D932D933C93A9ECB0E00D914E
:104040001C91A1EDB0E04D915C910E941334ADEC58
:10405000B0E04D935C9381E090E0AFECB0E08D93E5
:104060009C93ADECB0E04D915C91AFECB0E00D9164
:104070001C910417150718F011F00C946C20A0E7A0
:10408000B0E00D911D912D913C91A5E7B0E04D91CF
:104090005D916D917C910E942D3AA0E7B0E00D9367
:1040A0001D932D933D93A9ECB0E00D911D912D91A1
:1040B0003C9140E157E260E070E00E94323AA9ECA6
:1040C000B0E00D931D932D933D93AFECB0E00E94B3
:1040D000DC3310F40C94312088EE93E0A1EDB0E0D5
:1040E0008D939C93A9ECB0E00D911C91A1EDB0E0F3
:1040F0004D915C910E941334ADECB0E04D935C9314
:1041000081E090E0AFECB0E08D939C93ADECB0E03B
:104110004D915C91AFECB0E00D911C910417150727
:1041200018F011F00C94C120A0E7B0E00D911D91A2
:104130002D913C91A9E7B0E04D915D916D917C91FD
:104140000E942D3AA0E7B0E00D931D932D933D936F
:10415000A9ECB0E00D911D912D913C9148EE53E0FA
:1041600060E070E00E94323AA9ECB0E00D931D933C
:104170002D933D93AFECB0E00E94DC3310F40C942F
:10418000862084E690E0A1EDB0E08D939C93A9ECAD
:10419000B0E00D911C91A1EDB0E04D915C910E94B9
:1041A0001334ADECB0E04D935C9381E090E0AFEC64
:1041B000B0E08D939C93ADECB0E04D915C91AFEC91
:1041C000B0E00D911C910417150718F011F00C9434
:1041D0001621A0E7B0E00D911D912D913C91ADE726
:1041E000B0E04D915D916D917C910E942D3AA0E7D8
:1041F000B0E00D931D932D933D93A9ECB0E00D918C
:104200001D912D913C9144E650E060E070E00E94E9
:10421000323AA9ECB0E00D931D932D933D93AFEC92
:10422000B0E00E94DC3310F40C94DB208AE090E0D4
:10423000A1EDB0E08D939C93A9ECB0E00D911C91A1
:10424000A1EDB0E04D915C910E941334ADECB0E073
:104250004D935C9381E090E0AFECB0E08D939C9344
:10426000ADECB0E04D915C91AFECB0E00D911C91E4
:104270000417150718F011F00C946B21A0E7B0E0BB
:104280000D911D912D913C91A1E8B0E04D915D9172
:104290006D917C910E942D3AA0E7B0E00D931D93A3
:1042A0002D933D93A9ECB0E00D911D912D913C9182
:1042B0004AE050E060E070E00E94323AA9ECB0E0E1
:1042C0000D931D932D933D93AFECB0E00E94DC3332
:1042D00010F40C943021A9ECB0E08D919C91ADECE0
:1042E000B0E08D939C9381E090E0AFECB0E08D93D3
:1042F0009C93ADECB0E04D915C91AFECB0E00D91D2
:104300001C910417150718F011F00C94A221A0E7D6
:10431000B0E00D911D912D913C91A5E8B0E04D913B
:104320005D916D917C910E942D3AA0E7B0E00D93D4
:104330001D932D933D93AFECB0E00E94DC3310F45D
:104340000C947921089500E010E020E030E0A0E72F
:10435000B0E00D931D932D933C938D9A8C9A949875
:10436000A0E7B0E090E28D91983018F4392F9927AA
:1043700002C038E098508795959808F4959A000007
:104380000000949A000000009498000000003A9504
:1043900091F7992341F780E0809374008D9A8C9A6D
:1043A0009498A4E7B0E098E08D91983018F4392FF4
:1043B000992702C038E098508795959808F4959A07
:1043C00000000000949A0000000094980000000093
:1043D0003A9591F7992341F7969A00009698089597
:1043E000ECE0FAE70E944A39E5EDF0E0D190E08098
:1043F000FF2400270E9408380E94AF38EDE0F0E06B
:10440000A8EDB0E00E94DA3AE0E1FAE70E944A390A
:10441000E8EDF0E00E94E4370E94E038EDE0F0E0E3
:10442000A8EDB0E00E94DA3AE4E1FAE70E944A39E6
:10443000E8EDF0E00E94E4370E94EF38EDE0F0E0B4
:10444000A8EDB0E00E94DA3A0027A2E3B0E08C9138
:1044500083FB0EF401E041E0041711F00C945022AC
:10446000E8E1FAE70E944A39E8EDF0E00E94E4371B
:104470000E94EF38EDE0F0E0A8EDB0E00E94DA3AFB
:10448000E0EDF9E70E944A39E8EDF0E00E94E437F8
:104490000E945938EDE0F0E0A8EDB0E00E94DA3A71
:1044A000ECE1FAE70E944A39E8EDF0E00E94E437D7
:1044B0000E94AF38EDE0F0E0A8EDB0E00E94DA3AFB
:1044C000E0E2FAE70E944A39E8EDF0E00E94E437C2
:1044D0000E945938EDE0F0E0ACE0B1E00E94DA3A39
:1044E000A0E1B1E0E8EFF9E70E947439E0E1F1E022
:1044F000ACE0B1E00E947B3CEDE0F0E0A0EEB0E08B
:104500000E94DA3AE0EEF0E00E94E937E4E2FAE7EE
:104510000E9441390E945938EDE0F0E0A0EEB0E091
:104520000E94DA3AE0EEF0E00E94E937E4E2FAE7CE
:104530000E9441390E94EF38EDE0F0E0ACE0B1E0DC
:104540000E94DA3AE0EEF0E00E94E937E4E2FAE7AE
:104550000E9441390E94E038EDE0F0E0A0E1B1E0D6
:104560000E94DA3AE0E1F1E00E94E937ECE0F1E0A4
:104570000E94E4370E945938EDE0F0E0A4E1B1E098
:104580000E94DA3AE4E1F1E00E94273BEDE0F0E03E
:10459000A0E0B1E00E94DA3AE8E2FAE70E944A3984
:1045A000E3EDF0E0D190E080FF2400270E9408387E
:1045B0000E94AF38EDE0F0E0ACEDB0E00E94DA3AF6
:1045C000ECE2FAE70E944A39ECEDF0E00E94E437B1
:1045D0000E945938EDE0F0E0ACE0B1E00E94DA3A38
:1045E000ECE0F1E00E94463BEDE0F0E0A4EEB0E04C
:1045F0000E94DA3AECE0F1E00E949D3CEDE0F0E050
:10460000A8EEB0E00E94DA3AE0EEF0E00E94E9376E
:10461000E4EEF0E00E94E4370E94AF38EDE0F0E015
:10462000ACEEB0E00E94DA3AE0EEF0E00E94E9374A
:10463000E8EEF0E00E94E4370E94AF38EDE0F0E0F1
:10464000A0EFB0E00E94DA3AECEEF0E00E94E93729
:10465000E4E2FAE70E9441390E94E038EDE0F0E040
:10466000ACE0B1E00E94DA3AECE0F1E00E94E93718
:10467000ECE0F1E00E94E4370E94AF38EDE0F0E0BA
:10468000A4E0B1E00E94DA3AE0EFF0E00E94E937FE
:10469000E0EFF0E00E94E4370E94AF38EDE0F0E098
:1046A000A8E0B1E00E94DA3AE8E0F1E00E94E937E0
:1046B000E4E0F1E00E94E4370E94EF38EDE0F0E042
:1046C000ACE0B1E00E94DA3AE0EFF0E00E94E937B6
:1046D000E0EDF9E70E9441390E94AF38EDE0F0E0EB
:1046E000A0E1B1E00E94DA3AECE0F1E00E94E937A3
:1046F000E0E1F1E00E94E4370E945938EDE0F0E09B
:10470000A4E1B1E00E94DA3AECEDF9E70E944A39FF
:10471000E4E1F1E00E94E4370E94AF38EDE0F0E020
:10472000ACE0B1E00E94DA3AECE0F1E00E94273B15
:10473000EDE0F0E0A4EFB0E00E94DA3AECEEF0E059
:104740000E94E937ECEEF0E00E94E4370E94AF38B7
:10475000EDE0F0E0ACE0B1E00E94DA3AECE0F1E04C
:104760000E94E937E4E2FAE70E9441390E94E0380A
:10477000EDE0F0E0A0E1B1E00E94DA3AE8E0F1E03B
:104780000E94E937E0E1F1E00E94E4370E94E0385E
:10479000EDE0F0E0ACE0B1E00E94DA3AE8E0F1E010
:1047A0000E94E937E4E0F1E00E94E4370E94EF382C
:1047B000EDE0F0E0A0E1B1E00E94DA3AE0E1F1E002
:1047C0000E94E937ECE0F1E00E94E4370E9459389A
:1047D000EDE0F0E0A4E1B1E00E94DA3AECEDF9E7B7
:1047E0000E944A39E4E1F1E00E94E4370E94AF38C8
:1047F000EDE0F0E0ACE0B1E00E94DA3AECE0F1E0AC
:104800000E94273BEDE0F0E0A8EFB0E00E94DA3A2A
:10481000E8EFF0E00E94E937E8EFF0E00E94E437CB
:104820000E94AF38EDE0F0E0ACE0B1E00E94DA3A8F
:10483000E4EFF0E00E94E937E4EFF0E00E94E437B3
:104840000E94AF38EDE0F0E0A0E1B1E00E94DA3A7A
:10485000E0E1F1E00E94E937ECE0F1E00E94E437AA
:104860000E94EF38EDE0F0E0A4E1B1E00E94DA3A16
:10487000E4E1F1E00E94C23CEDE0F0E0ACEFB0E03A
:104880000E94DA3A0895ECE0FAE70E944A39E5ED31
:10489000F0E0D190E080FF2400270E9408380E94B9
:1048A000AF38EDE0F0E0A8EDB0E00E94DA3AE0E1E8
:1048B000FAE70E944A39E8EDF0E00E94E4370E94EE
:1048C000E038EDE0F0E0A8EDB0E00E94DA3AE4E193
:1048D000FAE70E944A39E8EDF0E00E94E4370E94CE
:1048E000EF38EDE0F0E0A8EDB0E00E94DA3A002702
:1048F000A2E3B0E08C9183FB0EF401E041E00417E9
:1049000011F00C94A324E8E1FAE70E944A39E8ED9B
:10491000F0E00E94E4370E94EF38EDE0F0E0A8ED0F
:10492000B0E00E94DA3AE0EDF9E70E944A39E8ED9A
:10493000F0E00E94E4370E945938EDE0F0E0A8ED85
:10494000B0E00E94DA3AECE1FAE70E944A39E8ED79
:10495000F0E00E94E4370E94AF38EDE0F0E0A8ED0F
:10496000B0E00E94DA3A0027A2E3B0E08C9183FB2A
:104970000EF401E040E0041711F00C942B25E0E266
:10498000FAE70E944A39E8EDF0E00E94E4370E941D
:104990005938EDE0F0E0ACE0B1E00E94DA3AA0E195
:1049A000B1E0E8EFF9E70E947439E0E1F1E0ACE052
:1049B000B1E00E947B3CEDE0F0E0A0EEB0E00E94B0
:1049C000DA3AE0EEF0E00E94E937E4E2FAE70E942A
:1049D00041390E945938EDE0F0E0A0EEB0E00E94CD
:1049E000DA3AE0EEF0E00E94E937E4E2FAE70E940A
:1049F00041390E94EF38EDE0F0E0ACE0B1E00E9418
:104A0000DA3AE0EEF0E00E94E937E4E2FAE70E94E9
:104A100041390E94E038EDE0F0E0A0E1B1E00E9411
:104A2000DA3AE0E1F1E00E94E937ECE0F1E00E94DF
:104A3000E4370E945938EDE0F0E0A4E1B1E00E94D3
:104A4000DA3AE4E1F1E00E94273BEDE0F0E0A0E09B
:104A5000B1E00E94DA3AE8E2FAE70E944A39E3ED6F
:104A6000F0E0D190E080FF2400270E9408380E94E7
:104A7000AF38EDE0F0E0ACEDB0E00E94DA3A089536
:104A800000916800013011F00C947125A5E6B0E0AA
:104A90008C918F5F8C9300916500063010F40C941C
:104AA000542581E0809365005A924A928AE090E012
:104AB000A42DB52D8D939C9382E00E94C9335A9208
:104AC0004A9281E0A42DB52D8C9381E00E94C933D8
:104AD0000E94142E249683E00E94C53380E08093C8
:104AE000660000916800033011F00C94BE2500911F
:104AF0006500013011F00C94822581E080936600FE
:104B00000C94A425023011F00C948B2585E0809341
:104B100066000C94A425033011F00C94942584E0D5
:104B2000809366000C94A425043011F00C949D250C
:104B300088E0809366000C94A425053011F00C9455
:104B4000A4258AE0809366005A924A9288E290E017
:104B5000A42DB52D8D939C9382E00E94C9335A9267
:104B60004A9281E0A42DB52D8C9381E00E94C93337
:104B70000E94142E249683E00E94C53300916800A1
:104B8000023011F00C940B2600916500013011F0F9
:104B90000C94CF2582E0809366000C94F1250230BE
:104BA00011F00C94D82586E0809366000C94F125D2
:104BB000033011F00C94E12583E0809366000C949F
:104BC000F125043011F00C94EA2587E0809366000B
:104BD0000C94F125053011F00C94F12589E08093B7
:104BE00066005A924A928EE190E0A42DB52D8D93E5
:104BF0009C9382E00E94C9335A924A9282E0A42D8B
:104C0000B52D8C9381E00E94C9330E94142E249606
:104C100083E00E94C53300916600013011F00C94CE
:104C20004E260091C2000A3011F00C9433265A929D
:104C30004A9284E690E0A42DB52D8D939C9382E05A
:104C40000E94C9335A924A9283E0A42DB52D8C93C9
:104C500081E00E94C9330E94142E249683E00E94B2
:104C6000C5330C944E26A2ECB0E08C918F5F8C93F0
:104C7000E8E8FDE5A2ECB0E08C919927A1E9B0E06D
:104C80000E947F39E4EBFDE5A2ECB0E08C9199271E
:104C90000E948639ADEBB0E00E9467370091660054
:104CA000023011F00C9491260091C200003011F0F6
:104CB0000C9476265A924A9284E690E0A42DB52D63
:104CC0008D939C9382E00E94C9335A924A9283E06A
:104CD000A42DB52D8C9381E00E94C9330E94142E1F
:104CE000249683E00E94C5330C949126A2ECB0E098
:104CF0008C9181508C93E8E8FDE5A2ECB0E08C91BA
:104D00009927A1E9B0E00E947F39E4EBFDE5A2EC30
:104D1000B0E08C9199270E948639ADEBB0E00E94FB
:104D2000673700916600033011F00C946D27809175
:104D3000EF018F7D8093EF010091C3000B3011F0E4
:104D40000C94BE265A924A9284E690E0A42DB52D8A
:104D50008D939C9382E00E94C9335A924A9283E0D9
:104D6000A42DB52D8C9381E00E94C9330E94142E8E
:104D7000249683E00E94C5330C946D270091C300F4
:104D800041E0040FA4ECB0E00C93ECEEFDE5A4ECE4
:104D9000B0E08C919927A9EBB0E00E947F39A9EB94
:104DA000B0E00D911D912D913C9142E050E060E00A
:104DB00070E00E946534A5EAB0E04D935D936D9379
:104DC0007D93A9E8B0E00D911D912D913C91A5EA4C
:104DD000B0E04D915D916D917C910E94323AA5EACF
:104DE000B0E00D931D932D933D93A9EBB0E00D9191
:104DF0001D912D913C9142E050E060E070E00E94F6
:104E00006534A9EAB0E04D935D936D937D93A9E875
:104E1000B0E00D911D912D913C91A9EAB0E04D912A
:104E20005D916D917C910E942D3AA9EAB0E00D93BD
:104E30001D932D933D9344E650E060E070E0A5EAB9
:104E4000B0E00D911D912D913C910E94373A80E088
:104E50000CF481E08F9348EE5DEF60E070E0A9EA2A
:104E6000B0E00D911D912D913C910E94373A80E068
:104E700014F009F081E09F91892B882311F40C94A0
:104E80005D275A924A9284E690E0A42DB52D8D9329
:104E90009C9382E00E94C9335A924A9283E0A42DE7
:104EA000B52D8C9381E00E94C9330E94142E249664
:104EB00083E00E94C5330C946D278091C4008093D9
:104EC000C300A9EBB0E00D911D912D913C91ADE88F
:104ED000B0E00D931D932D933C9300916600043038
:104EE00011F00C9449280091C300003011F00C948B
:104EF0009A278091EF0180628093EF015A924A9243
:104F000088EC90E0A42DB52D8D939C9382E00E94B7
:104F1000C9335A924A9284E0A42DB52D8C9381E036
:104F20000E94C9330E94142E249683E00E94C53348
:104F30000C9449280091C30041E0041BA4ECB0E0AC
:104F40000C93ECEEFDE5A4ECB0E08C919927A9EB75
:104F5000B0E00E947F39A9EBB0E00D911D912D9139
:104F60003C9142E050E060E070E00E946534A5EAC8
:104F7000B0E04D935D936D937D93A9E8B0E00D9102
:104F80001D912D913C91A5EAB0E04D915D916D91FF
:104F90007C910E94323AA5EAB0E00D931D932D93C7
:104FA0003D93A9EBB0E00D911D912D913C9142E014
:104FB00050E060E070E00E946534A9EAB0E04D93F3
:104FC0005D936D937D93A9E8B0E00D911D912D91B6
:104FD0003C91A9EAB0E04D915D916D917C910E9468
:104FE0002D3AA9EAB0E00D931D932D933D9344E62D
:104FF00050E060E070E0A5EAB0E00D911D912D91C8
:105000003C910E94373A80E00CF481E08F9348EEA7
:105010005DEF60E070E0A9EAB0E00D911D912D9187
:105020003C910E94373A80E014F009F081E09F91B2
:10503000892B882311F40C9439285A924A9284E6D9
:1050400090E0A42DB52D8D939C9382E00E94C933EE
:105050005A924A9283E0A42DB52D8C9381E00E9450
:10506000C9330E94142E249683E00E94C5330C9409
:1050700049288091C4008093C300A9EBB0E00D9152
:105080001D912D913C91ADE8B0E00D931D932D93B2
:105090003C9300916600053011F00C94F9280091C2
:1050A0006700053011F00C947D28E0E3FAE70E94D8
:1050B0004A39E8E1F1E00E94E4370E94EF38EDE080
:1050C000F0E0A8E1B1E00E94DA3AE8E1F1E00E9404
:1050D000E437E4E2FAE70E944A390E94533918F0B3
:1050E00011F00C9475280C947B28A8E1B1E0E4E25F
:1050F000FAE70E9474390C94F928ADE8B0E00D91FC
:105100001D912D913C9142E050E060E070E00E94E2
:105110006534A5EAB0E04D935D936D937D93A9E866
:10512000B0E00D911D912D913C91A5EAB0E04D911B
:105130005D916D917C910E942D3AA5EAB0E00D93AE
:105140001D932D933D93A5EAB0E00D911D912D91F6
:105150003C91A1E9B0E04D915D916D917C910E94EF
:105160002D3AA5EAB0E00D931D932D933D9348EEA3
:105170005DEF60E070E0A5EAB0E00D911D912D912A
:105180003C910E94373A1CF011F00C94C9280C9401
:10519000E5285A924A9284E690E0A42DB52D8D938D
:1051A0009C9382E00E94C9335A924A9283E0A42DD4
:1051B000B52D8C9381E00E94C9330E94142E249651
:1051C00083E00E94C5330C94F928A9E8B0E00D9162
:1051D0001D912D913C91A1E9B0E04D915D916D91B2
:1051E0007C910E942D3AA9E8B0E00D931D932D9378
:1051F0003D9300916600063011F00C94A4290091B3
:105200006700053011F00C942A29E0E3FAE70E94C8
:105210004A39E8E1F1E00E94E4370E94E038EDE02D
:10522000F0E0A8E1B1E00E94DA3AE8E1F1E00E94A2
:10523000E437E4E3FAE70E944A390E94533910F058
:105240000C942829A8E1B1E0E4E3FAE70E9474395C
:105250000C94A429ADE8B0E00D911D912D913C91E5
:1052600042E050E060E070E00E946534A5EAB0E002
:105270004D935D936D937D93A9E8B0E00D911D91E1
:105280002D913C91A5EAB0E04D915D916D917C919D
:105290000E94323AA5EAB0E00D931D932D933D9301
:1052A000A5EAB0E00D911D912D913C91A1E9B0E0EE
:1052B0004D915D916D917C910E94323AA5EAB0E0EA
:1052C0000D931D932D933D9344E650E060E070E014
:1052D000A5EAB0E00D911D912D913C910E94373AC5
:1052E0000CF402C00C9490295A924A9284E690E001
:1052F000A42DB52D8D939C9382E00E94C9335A92C0
:105300004A9283E0A42DB52D8C9381E00E94C9338D
:105310000E94142E249683E00E94C5330C94A42985
:10532000A9E8B0E00D911D912D913C91A1E9B0E06B
:105330004D915D916D917C910E94323AA9E8B0E067
:105340000D931D932D933D9300916600073011F04E
:105350000C945E2AADE8B0E00D911D912D913C9129
:1053600042E050E060E070E00E946534A5EBB0E000
:105370004D935D936D937D93A9E8B0E00D911D91E0
:105380002D913C91A5EBB0E04D915D916D917C919B
:105390000E94323AADEAB0E00D931D932D933D93F8
:1053A000ADEAB0E00D911D912D913C91A1E9B0E0E5
:1053B0004D915D916D917C910E94323AADEAB0E0E1
:1053C0000D931D932D933D9344E650E060E070E013
:1053D000ADEAB0E00D911D912D913C910E94373ABC
:1053E0000CF402C00C94102A5A924A9284E690E07F
:1053F000A42DB52D8D939C9382E00E94C9335A92BF
:105400004A9283E0A42DB52D8C9381E00E94C9338C
:105410000E94142E249683E00E94C5330C945E2AC9
:10542000A9E8B0E00D911D912D913C91A5EBB0E064
:105430004D915D916D917C910E942D3AA1EBB0E070
:105440000D931D932D933D93A1EBB0E00D911D9114
:105450002D913C91ADEAB0E04D915D916D917C91C3
:105460000E94323AADE8B0E00D931D932D933D9329
:10547000ADE8B0E00D911D912D913C9142E050E0DE
:1054800060E070E00E946534A5EBB0E04D935D9361
:105490006D937D93ADEAB0E00D911D912D913C91FE
:1054A000A5EBB0E04D915D916D917C910E942D3AFC
:1054B000A9E8B0E00D931D932D933D9300916600F4
:1054C000083011F00C941C2BADE8B0E00D911D914B
:1054D0002D913C9142E050E060E070E00E94653424
:1054E000A5EBB0E04D935D936D937D93A9E8B0E09B
:1054F0000D911D912D913C91A5EBB0E04D915D91E9
:105500006D917C910E94323AADEAB0E00D931D930B
:105510002D933D93ADEAB0E00D911D912D913C91FD
:10552000A1E9B0E04D915D916D917C910E942D3A81
:10553000ADEAB0E00D931D932D933D93A9E8B0E043
:105540004D915D916D917C91ADEAB0E00D911D9111
:105550002D913C910E94373A1CF011F00C94B22A24
:105560000C94CE2A5A924A9284E690E0A42DB52D4E
:105570008D939C9382E00E94C9335A924A9283E0B1
:10558000A42DB52D8C9381E00E94C9330E94142E66
:10559000249683E00E94C5330C941C2BA9E8B0E04C
:1055A0000D911D912D913C91A5EBB0E04D915D9138
:1055B0006D917C910E942D3AA1EBB0E00D931D936B
:1055C0002D933D93A1EBB0E00D911D912D913C9158
:1055D000ADEAB0E04D915D916D917C910E94323ABF
:1055E000ADE8B0E00D931D932D933D93ADE8B0E091
:1055F0000D911D912D913C9142E050E060E070E0F2
:105600000E946534A5EBB0E04D935D936D937D935F
:10561000ADEAB0E00D911D912D913C91A5EBB0E06C
:105620004D915D916D917C910E942D3AA9E8B0E079
:105630000D931D932D933D9300916600093011F059
:105640000C94D82BADE8B0E00D911D912D913C91BB
:1056500042E050E060E070E00E946534A5EBB0E00D
:105660004D935D936D937D93A9E8B0E00D911D91ED
:105670002D913C91A5EBB0E04D915D916D917C91A8
:105680000E942D3AA1EBB0E00D931D932D933D9315
:10569000A1EBB0E00D911D912D913C91A1E9B0E0FD
:1056A0004D915D916D917C910E94323AA1EBB0E0F9
:1056B0000D931D932D933D93A9E8B0E04D915D911D
:1056C0006D917C91A1EBB0E00D911D912D913C91DC
:1056D0000E94373A0CF402C00C948A2B5A924A92D8
:1056E00084E690E0A42DB52D8D939C9382E00E94DA
:1056F000C9335A924A9283E0A42DB52D8C9381E050
:105700000E94C9330E94142E249683E00E94C53360
:105710000C94D82BA9E8B0E00D911D912D913C91EE
:10572000A5EBB0E04D915D916D917C910E94323A74
:10573000ADEAB0E00D931D932D933D93A1EBB0E046
:105740000D911D912D913C91ADEAB0E04D915D918F
:105750006D917C910E94323AADE8B0E00D931D93BB
:105760002D933D93ADE8B0E00D911D912D913C91AD
:1057700042E050E060E070E00E946534A5EBB0E0EC
:105780004D935D936D937D93ADEAB0E00D911D91C6
:105790002D913C91A5EBB0E04D915D916D917C9187
:1057A0000E942D3AA9E8B0E00D931D932D933D93EF
:1057B000009166000A3011F00C94942CADE8B0E032
:1057C0000D911D912D913C9142E050E060E070E020
:1057D0000E946534A5EBB0E04D935D936D937D938E
:1057E000A9E8B0E00D911D912D913C91A5EBB0E0A1
:1057F0004D915D916D917C910E942D3AA1EBB0E0AD
:105800000D931D932D933D93A1EBB0E00D911D9150
:105810002D913C91A1E9B0E04D915D916D917C910C
:105820000E942D3AA1EBB0E00D931D932D933D9373
:1058300048EE5DEF60E070E0A1EBB0E00D911D91EE
:105840002D913C910E94373A1CF011F00C942A2CB7
:105850000C94462C5A924A9284E690E0A42DB52DE1
:105860008D939C9382E00E94C9335A924A9283E0BE
:10587000A42DB52D8C9381E00E94C9330E94142E73
:10588000249683E00E94C5330C94942CA9E8B0E0E0
:105890000D911D912D913C91A5EBB0E04D915D9145
:1058A0006D917C910E94323AADEAB0E00D931D9368
:1058B0002D933D93A1EBB0E00D911D912D913C9165
:1058C000ADEAB0E04D915D916D917C910E94323ACC
:1058D000ADE8B0E00D931D932D933D93ADE8B0E09E
:1058E0000D911D912D913C9142E050E060E070E0FF
:1058F0000E946534A5EBB0E04D935D936D937D936D
:10590000ADEAB0E00D911D912D913C91A5EBB0E079
:105910004D915D916D917C910E942D3AA9E8B0E086
:105920000D931D932D933D93089580E0809368001F
:105930000027A3E3B0E08C9180FB0EF401E040E08F
:10594000041781E009F080E08F930027A3E3B0E023
:105950008C9181FB0EF401E040E0041781E009F036
:1059600080E09F91892B8F930027A0E3B0E08C917A
:1059700087FB0EF401E040E0041781E009F080E0CD
:105980009F91892B882311F40C94132E84E190E0CD
:105990000E94C2340027A3E3B0E08C9180FB0EF498
:1059A00001E040E0041781E009F080E08F930027D8
:1059B000A3E3B0E08C9181FB0EF401E040E004171A
:1059C00081E009F080E09F918923882311F40C94F1
:1059D0009E2DA7E6B0E08C918F5F8C9300916700BD
:1059E000053018F011F00C94F72C0C94FA2C81E08F
:1059F0008093670000916700013011F00C94092D2D
:105A00009398A1E3B1E0EEE9FBE70E9467370C94BD
:105A1000432D00916700023011F00C94182D9398DB
:105A2000A1E3B1E0E0EAFBE70E9467370C94432D65
:105A300000916700033011F00C94272D939AA1E395
:105A4000B1E0E2EAFBE70E9467370C94432D009136
:105A50006700043011F00C94362D9398A1E3B1E067
:105A6000E4EAFBE70E9467370C94432D009167003E
:105A7000053011F00C94432D9398A1E3B1E0E6EAD0
:105A8000FBE70E9467375A924A9288E7A42DB52D0A
:105A90008C9381E00E94C9335A924A9280E0A42DEF
:105AA000B52D8C9381E00E94C933E1E3F1E0FA93D4
:105AB000EA930E946A13269682E00E94C5335A92A6
:105AC0004A9285E090E0A42DB52D8D939C9382E0C1
:105AD0000E94C9335A924A9281E0A42DB52D8C932D
:105AE00081E00E94C9330E94142E249683E00E9414
:105AF000C53384E690E00E94C2340027A3E3B0E0FF
:105B00008C9180FB0EF401E041E0041781E009F084
:105B100080E08F930027A3E3B0E08C9181FB0EF42B
:105B200001E041E0041781E009F080E09F918923C2
:105B3000882311F40C947D2D0C94132E0027A3E3DD
:105B4000B0E08C9180FB0EF401E040E0041711F00E
:105B50000C94D12DA1E3B1E0E8EAFBE70E9467379E
:105B60005A924A9288E7A42DB52D8C9381E00E9429
:105B7000C9335A924A9280E0A42DB52D8C9381E0CE
:105B80000E94C933E1E3F1E0FA93EA930E946A13B9
:105B9000269682E00E94C53382E0809368000C94D0
:105BA000132E0027A3E3B0E08C9181FB0EF401E0FB
:105BB00040E0041711F00C94042EA1E3B1E0EAEAEE
:105BC000FBE70E9467375A924A9288E7A42DB52DC9
:105BD0008C9381E00E94C9335A924A9280E0A42DAE
:105BE000B52D8C9381E00E94C933E1E3F1E0FA9393
:105BF000EA930E946A13269682E00E94C53383E0EE
:105C0000809368000C94132E0027A0E3B0E08C91E1
:105C100087FB0EF401E040E0041711F00C94132E02
:105C200081E080936800089581E090E0ABE6B0E009
:105C30008D939C93AA81BB814D915C91ABE6B0E0C2
:105C40000D911C910417150718F011F00C94432EB8
:105C500082B394E0892782BBA881B9818C9199276E
:105C60000E94C23482B394E0892782BBA881B981A3
:105C70008C9199270E94C234ABE6B0E00E94DC33DD
:105C800010F40C941A2E92980895939A82E390E05F
:105C90000E94C234939882E390E00E94C234939AA7
:105CA00082E390E00E94C234939882E390E00E94E5
:105CB000C234939A939882E390E00E94C23408958C
:105CC000F894FFCF588A6042158C0E427502B84195
:105CD000D8F07641C4423041C18B07417F6ADF4032
:105CE000D786C140C251AC4005179B4086C98B4046
:105CF000D39F7B404278624083A34C40F4893A4072
:105D0000C53D2C40E6742140B79C194098FA1340D9
:105D1000E6CB0F404E620C40A835094029ED054006
:105D2000B35E0240A110FD3F7906F53F3EEDEC3F2A
:105D30003815E53F5EBADD3F38F8D63F8AC8D03F18
:105D40009E07CB3F5183C53F1B0DC03FC68ABA3F5C
:105D50008104B53F8BA6AF3FAEB6AA3F077CA63FF6
:105D6000B116A33F8F53A03F5A819D3F9560993F45
:105D70004547923FCDCC8C3F6666863F0AD7833F2E
:105D8000AE47813F0000803F010000000A00000094
:105D9000140000003200000064000000C800000091
:105DA000F4010000E8030000D007000088130000A1
:105DB000102700002020314B002031304B002032D2
:105DC000304B002035304B003130304B003230301A
:105DD0004B003530304B002020314D002020324D1B
:105DE000002020354D002031304D00000A00000019
:105DF000140000003200000064000000C800000031
:105E0000F4010000E8030000D00700008813000040
:105E100010270000204E000050C30000000810159D
:105E200008000304081000081F1F0800021F1F02BB
:105E30000000000000000001000000000404040055
:105E4000000B150900001D15120000101718000E98
:105E500011110E00091F0100000B151509000A1190
:105E6000150E00060A1F02001D15151200020D1561
:105E7000020010131418000A15150A000815160C54
:105E8000000F14140F001F15150A000E1111110038
:105E90001F11110E001F151111001F141010000EFC
:105EA000111517001F04041F00111F11000012110B
:105EB000111E001F040A11001F010101001F181804
:105EC0001F001F18061F000E11110E001F141408CA
:105ED000000E11130F001F141609000915151200EA
:105EE000101F1000001E01011E001C02011E001FD9
:105EF00003031F00110A061900110A0418001315E4
:105F0000151900111F0E04004080FF01AA0101C1F4
:105F1000E1F131F1E1C101AA0101C1AA02C141C10E
:105F2000AA01C18101AA010141F1AA02F141AA021B
:105F30004101AA010181C1AA01C141C1AA01C181D6
:105F400001AA0101C1AA02C141C1AA01C18101AADC
:105F50000101C1AA02C141C1AA01C18101AA020174
:105F600041AA0241C1AA01C18101AA3E01FFAA01C1
:105F7000FF00AA01001FAA021F021FAA021F00AAF7
:105F800001001FAA021F001FAA021F00AA02000F81
:105F90001FAA011F10AA021000AA01000F1FAA01C8
:105FA0001F1213AA01130300AA01001FAA021F0057
:105FB0001FAA021F00AA01001FAA021F001FAA0297
:105FC0001F00AA01000C1EAA011E121FAA021F0018
:105FD000AA3E00FFAA01FF00AA0A00E0F0F818F8A4
:105FE000F0E000AA0100E0AA02E020E0AA01E0C07F
:105FF00000AA020020AA0220E0AA01E0C000AA0133
:106000000008AA0108F8AA02F800AA0300E0AA0200
:10601000E000E0AA02E000AA0100C0E0AA01E0203E
:10602000AA032000AA0100C0E0AA01E020E0AA0122
:10603000E0C000AA0100E0AA02E0C060AA0260007D
:10604000AA0A00F8AA02F820E0AA01E0C000AA010A
:1060500000E0AA02E000E0AA02E000AA1100FFAA04
:1060600001FF00AA0A000FAA020F010FAA020F00E7
:10607000AA01000FAA020F000FAA020F00AA010036
:10608000060FAA010F090FAA020F00AA010008AA11
:1060900001080FAA020F08AA01080040474F6F78B5
:1060A0003F1F0700AA01000809AA02090FAA010F51
:1060B0000600AA0100070FAA010F09AA02090100A0
:1060C000AA01000FAA020F00AA0E000FAA020F08D1
:1060D0000FAA010F070040474F6F783F1F0700AA24
:1060E0001100FFAA01FF00AA0A008040AA01402077
:1060F00010AA031008AA030810AA03102040AA013E
:10610000408000AA5E00FFAA01FF00AA0700C03C71
:10611000020100AA0100040AAA010A0400AA01005F
:10612000F8AA01F800AA0100040AAA010A0400AAB8
:10613000010001023CC000AA06001E3E3361AA0114
:106140006141C3C78600AA0200FFAA01FF21AA037A
:1061500021233F1E00AA03000111191D1733E1C0BE
:1061600000AA02001E3E3361AA016141C3C7860036
:10617000AA020007FFF800C0FC3FAA013FFCC000D4
:10618000F8FF0700AA0900FFAA01FF00AA0A00FF02
:10619000AA01FF00AA0700033C408000AA010030CA
:1061A00020C08000AA01001FAA011F00AA010080D0
:1061B000C0203000AA010080403C0300AA06000471
:1061C0000C18AA011810AA0210180F0700AA010043
:1061D0001FAA011F00AA0900060E1810AA01101814
:1061E0001C0F0700AA0200040C18AA011810AA022A
:1061F00010180F0700AA03001FAA021F0300AA011C
:1062000000031FAA021F0100AA0200060E18AA011D
:106210001810AA0110180C0F0700AA0A00FFAA0103
:10622000FF80AA0A808182AA01828488AA028889C2
:1062300091AA03918988AA02888482AA0182818016
:10624000AA5E80FF4080FF01AA1A0105AA02050983
:10625000AA030911AA031121AA042141AA03418119
:10626000AA038101AA01018141AA01418101AA4138
:106270000181C141FFAA01FF00AA0C00F010AA0190
:1062800010D050AA0C50D010AA0110F000AA100093
:1062900001AA01010307AA0107030102AA020204DD
:1062A000AA050408AA050810AA041020AA0520407F
:1062B000AA054080AA048040AA034020AA03201017
:1062C000AA031008AA030804AA030402AA030201ED
:1062D000AA020100010203FFAA01FF00AA0C00FFAD
:1062E00000AA0100FF00AA0C00FF00AA0100FF00A5
:1062F000AA3800FF00AA2100FFAA01FF00AA05009A
:10630000FC04AA05040704AA010405AA090565AA54
:10631000046564AA01646764AA026404AA0104FC17
:106320002010AA011008AA010804AA010402AA0266
:106330000201AA080102AA0102041820C000AA1939
:1063400000FF00AA2100FFAA01FF00AA0400C04725
:1063500044AA1F44C700AA1800033CC000AA0B00AF
:10636000C040AA09407F40AA0940C000AA1600FF09
:10637000AA01FF00AA0400FF80AA0080AA0080AA48
:106380000080AA0080AA0080AA0080AA0080AA003B
:1063900080AA0080AA0080AA0080AA0080AA0080AB
:1063A000AA0080AA0080AA0080FF00AA1A000F108D
:1063B00020AA012040AA024080AA0580FF00FF0019
:1063C000AA0100E01886611806FF00806018866147
:1063D0001806FF00FF00AA1600FFAA01FF00AA0B83
:1063E00000C0E0AA01E020AA032000AA0100C0E04A
:1063F000AA01E020E0AA01E0C000AA0100E0AA0290
:10640000E0C060AA026000AA010020AA0120ECAA54
:1064100002EC00AA040020AA0220E0AA01E0C000C9
:10642000AA010008AA0108F8AA02F800AA11003F70
:10643000202F2C2328262120AA02202F262128269F
:1064400021AA0221222F203F00AA1600FFAA01FF45
:1064500080AA0B808889AA02898FAA018F8680AAC8
:106460000180878FAA018F89AA02898180AA018071
:106470008FAA028F80AA058088AA01888FAA028F1E
:1064800088AA018880AA0180868FAA018F898FAA95
:10649000028F80AA018088AA01888FAA028F88AA09
:1064A000018880AA3D80FF004080FFAA12FFF3C34D
:1064B0000F3FFFAA02FF3F0FC3F3FF03AA0103C769
:1064C0008F3F7FFFAA01FF03AA0103FFAA02FF7FFC
:1064D0000F83F3830F7FFFAA06FF03AA0103C30FF5
:1064E0007FFF7F0FC303AA0103FFAA02FF7F0F8371
:1064F000F3830F7FFFAA02FFF3E3871F3F1F87E3AA
:10650000F3FFAA02FF3F1FC703AA0103FFAA31FF3F
:10651000FEF8C1C7C1F8FEFFAA02FFC0AA01C0FF72
:10652000AA01FFFEFCF1E3C0AA01C0FFDFC3E0F84F
:10653000F9AA02F9F8E0C3DFFFAA04FFC0AA01C06C
:10654000FFFCE0C3E0FCFFC0AA01C0FFDFC3E0F82E
:10655000F9AA02F9F8E0C3DFFFCFC7E1F8FCF8E1E0
:10656000C7CFFFF1F0F2F3AA01F3C0AA01C0F3FF15
:10657000AA24FF07AA0107E7AA05E7FFAA01FF0768
:10658000AA0107E7AA04E7470F1FFFAA01FF07AA0E
:106590000107E7AA06E7FFAA01FF07AA0107E7AA82
:1065A00006E7FFAA05FF3FAA013FFFAA02FF3FAA95
:1065B000013FFFAA02FF7F3FAA023F7FFFAA02FF1F
:1065C0003FAA013F7F3FAA013FFF7F3FAA043F7FD1
:1065D000FFAA01FF27AA0127FFAA02FF7F3FAA0304
:1065E0003F7FFFAA02FF3FAA013F7F3FAA033F7FF1
:1065F000FFAA18FF80AA0180FCAA04FCFFAA02FFE0
:1066000080AA0180FCAA02FCF8F0C2869FBFFF802E
:10661000AA01809CAA069CFFAA01FF80AA01809C77
:10662000AA069CFFAA05FFFEF0818F81F0FEFFAA5B
:1066300001FFE0C08999AA0199C8E8FFAA01FF807B
:10664000AA0180FEFFAA02FFCC8899919382C6FF1F
:10665000AA01FF80AA0180FFAA01FFE0C08E9FAAC5
:10666000019F8EC0E0FFAA01FF80AA0180FEFFAA61
:1066700002FF80AA0180FFAA94FFC7BBAA02BB7BCE
:10668000AA017BE7FFAA01FF037BAA047B87FFF730
:10669000FBBBAA02BB47FFAA01FFC7BBAA02BB7B89
:1066A000AA017BE7FFF38F7FFF7F87FB877FFF7F59
:1066B0008FF3FFAA03FF03FFAA06FF473BBBC7FFF9
:1066C000AA07FFC7BBAA02BB7BAA017BE7FFAA01FF
:1066D000FF037BAA047B87FF47BBAA03BB47FFAA34
:1066E00001FF03F7CF3FFFAA01FF03FFFBAA02FB55
:1066F00003FBAA02FBFF03BFAA04BF03FFAA09FF13
:10670000F9F7AA04F7F8FFAA01FFF0FFAA06FFFBBA
:10671000F7AA03F7F8FFAA01FFF9F7AA04F7F8FFB1
:10672000AA02FFFCF3FCFFAA02FFFCF3FCFFAA0194
:10673000FFF9F7AA02F7F8FFAA05FFF8F7AA01F791
:10674000F6F9FBF4F7FFAA04FFF9F7AA04F7F8FF3C
:10675000AA01FFF0FFAA06FFF8F7AA03F7F8FFAABD
:1067600001FFF0FFAA02FFFCFBF0FFAA03FFF0FF0E
:10677000AA03FFF0FFAA04FFF0FFAA84FF008E2EF9
:106780009F2E0895E82DF92D0895481A8827580A54
:106790000895480E8827581E08950D911D912D913A
:1067A0003C9181E0080F8827181F281F381F3C9351
:1067B0002E931E930E930895ED91FC91EF5FFF4F82
:1067C000FC93EE930895ED91FC91E150F040FC9321
:1067D000EE93089500FC10D0089503D024D001F862
:1067E000F9CF0024E89457FF02C009D0689400F85C
:1067F0000BD010F80124089502D009D008955095C7
:1068000040954F5F5F4F0895E89417FF08950095F6
:1068100010950F5F1F4F6894089599231AF480957F
:10682000909501960895352F242FE894452B11F467
:1068300068940895512F402F0027112780E1440FBD
:10684000551F001F111F021B130B416018F4020F8C
:10685000131F4E7F8A9599F708958F938D91882302
:10686000E9F711978F910895AAE6B7E018D088301C
:1068700091F08D3039F03323C9F38D933A9563FE4F
:1068800017D0F4CF63FC04C08DE012D08AE010D0A2
:1068900088278C9308950CD011973395E7CF5F9B91
:1068A000FECF8CB108958D9103D03A95E1F708950C
:1068B0005D9BFECF8CB9089588EE93E063D031974D
:1068C000D9F7089500FC05D0089530D005D001F81F
:1068D000F9CF37D03FD00895842F952FA62FB72F0B
:1068E000E894452B462B472B11F468940895402FCC
:1068F000512F622F732F0027112722273327F0E211
:10690000440F551F661F771F001F111F221F331FC3
:10691000081B190B2A0B3B0B416028F4080F191FA9
:106920002A1F3B1F4E7FFA9559F708950024E894DB
:1069300077FF02C006D0689400F809D010F801244F
:10694000089512D04F5F5F4F6F4F7F4F0895E894C7
:1069500037FF089500951095209530950F5F1F4FD4
:106960002F4F3F4F689408954095509560957095CE
:1069700008953197F1F70895689462F80895E894BE
:1069800062F80895EF93FF93EE27E82BE92B31F09F
:10699000EDECFAE03197F1F70197D1F7FF91EF9124
:1069A00008955A924A92480E8827581E08958DE2FB
:1069B00007FD8D938F2D881F802F881F8F57082FDD
:1069C0006894F7F8802F87FF15C080958395082F6E
:1069D00080E38D938EE28D93802F815228F080E3A7
:1069E0008D9399279C93089544270A95802F09F148
:1069F00096D01FC0805230F09EE49D9381E48D9329
:106A00009D93EFCF4427DF92EF92FF920F938FE198
:106A1000801B11F0082F83D089D09EE29D930F91A7
:106A2000FF90EF90DF9044270395003209F4D7CF11
:106A30002BD03F93EEEBFAE638E12F2D1E2D0D2DD6
:106A4000FF24EE24DD244427000F111F221FA8F489
:106A50002F923F920E943D39102C0E943D39202CEC
:106A60000E943D39302C0E943D393197410DD21C96
:106A7000E31CF01C3F902F9001C0339631963A955D
:106A800019F73F9107D0AFCFDD0CEE1CFF1C0A9524
:106A9000D9F70895002719E058D08F93802B11F073
:106AA000039501C08F911A95B9F7802F882309F4B7
:106AB00096CF8F91805D8D930A95D9F792CF00651F
:106AC000CD1D80B2E60E40597307A0ACB90350D675
:106AD000DC01286BEE0094357700CA9A3B0065CD47
:106AE0001D00B2E60E0059730700ACB90300D6DCF6
:106AF00001006BEE0000357700009A3B0000CD1DD1
:106B00000000E60E000073070000B9030000DC017E
:106B10000000EE000000770000003B000000F6944B
:106B2000E794D79447950A95D1F7089500270DD09B
:106B30008F9303958F2D8E298D29842BC1F78F91EB
:106B4000805D8D930A95D9F74CCF1F930F93002743
:106B500010E2440FDD1CEE1CFF1C001F802F9AE08A
:106B6000890B10F0082F43951A9599F7802F0F91F4
:106B70001F91089520931D0330931E0340931F031C
:106B800050932003089520911D0330911E034091DE
:106B90001F03509120030895442719D0AD98AC9A53
:106BA000AA9884E699270E94C2349FEF97BBAD9ABA
:106BB00033D014FCFDCF02D04FEF09D08FE310D0BB
:106BC00080EC0ED080E40CD088EB0AD008954034DD
:106BD00020F0AF9AAE9840540895AE9AAF980895B9
:106BE000AB9801C0AB9AEF93FF93EAE0F0E00E940C
:106BF000B934FF91EF9188BBAC98AA9A00000000CD
:106C00000000000000000000000000000000000084
:106C100000000000AA980895AB9804D017FCFCCFA0
:106C20000895AB9A992797BB9FEF98BBEF93FF937B
:106C3000EAE0F0E00E94B934FF91EF91AC9AAA9A91
:106C4000EF93FF93E2E0F0E00E94B934FF91EF91FF
:106C500016B2AA9897BB08954427B9DF02D04FEF28
:106C6000B6DF00E080E4BCDF88EB800FB9DF10E422
:106C70008827B8DF1A95E1F70395083099F708954A
:106C8000EF93FF93509162005F9370906300E091E7
:106C90006000F09161000E943D39202D0E943D3935
:106CA000302D0E943D39002D31968052482F0E9490
:106CB000FF3AE40FF51F70926300732F4091630059
:106CC000509162001DD00E943D39802D509164008A
:106CD000552309F0809586DF5091630053955093BA
:106CE00063007A9559F75091620053955093620072
:106CF0002A9509F75F9150936200FF91EF910895F3
:106D00004A955A9564DF88EB850F6ADF80E4840F2B
:106D100067CF0F921F922F923F920F939F934F93A3
:106D2000052F48E00E940B3B082E4F91502F242E38
:106D3000352EE8DF76DF75DF422D532DE3DF802D22
:106D40000E9490390F91002311F0182A01C01922D6
:106D5000812D48DF0F913F902F901F900F90089545
:106D6000772321F0AA27BB270C94F53A0C943D39E0
:106D700011242224332479910E94B036002D48E05A
:106D80000E940B3B0A930E94B0360A920A920B8132
:106D900048E00E940B3B0B834C81F42E5B81B2DFF9
:106DA000131479F40E94B036202C802D8A3A39F0E1
:106DB0000E94B036802D8A3A39F031970DC0319655
:106DC0000BC01A9469F308C00E94B036802D882346
:106DD00011F4329701C0102C822D909164009923F8
:106DE00009F080958F934F2D5B818CDF8F91F39409
:106DF000F9DE89818A95898399F68B8183958B83C6
:106E0000888189838A818A958A8331F625960895B7
:106E1000AA24BB24FF24EC81EA80EE1AFF08FB8140
:106E2000298033242F1A330881E0EA14FA043CF451
:106E30002FEF3FEFE094F094E80EFA1C02C021E03F
:106E400033272A143A043CF46FEF7FEF20943094F8
:106E5000280E3A1C02C061E0772735D02E143F047B
:106E600014F009F017C0CE2CDF2CCC0CDD1C022C4A
:106E7000132C000C111C9A81E91761F0E20FA00C91
:106E8000B11CAE14BF0424F019F0F60FAC18BD0805
:106E90001AD0F1CFC22CD32CCC0CDD1C0E2C1F2C05
:106EA000000C111C9981F91711F425960895F60F1D
:106EB000A00CB11CA214B30424F019F0E20FAC181A
:106EC000BD0801D0EFCF4E2F5F2F988122CF0E94B7
:106ED0003D390D920020D9F70895369A3699FECFA4
:106EE000369A3699FECF84B195B1089599910027CD
:106EF000A90FB01F1197492F4A955E2F6F2FE89465
:106F000011274395203019F0C895802D01C080814C
:106F10008823B9F07C917723A1F0781739F40EF02B
:106F2000042F1395689411963196EBCF112321F01D
:106F3000411BA11B1127B10BE894E52FF62F1196E9
:106F4000E0CF882311F00027089508953DD09927B8
:106F500011278F2D880F80E8F82A802F881F08F4CA
:106F60001FEF41F08F57082F07FD04C0003240F09B
:106F70008FEF01C08827982FD82EE82EF82E09C051
:106F80008FE1801B082FF694E794D79497950A9584
:106F9000D1F7112351F09095D094E094F09481E0D2
:106FA000980F8827D81EE81EF81E0F2DFE2CED2CFA
:106FB000D92E0895D094E094F09491E0D90E9927B9
:106FC000E91EF91E10950895D190E190F19001917C
:106FD000089521913191419151910895102F90E898
:106FE000FF0C001F0927990FF7941078652F90E880
:106FF000440F551F5927990F479560780038089519
:10700000FF0C90E89027110F9795F794092F08959A
:10701000102FBD2CDE2CEF2CF02E11234AF4B0944F
:10702000D094E094F0949FEFB91AD90AE90AF90ACA
:107030000EE1FF2039F4FE2CED2CDB2CBB24085094
:10704000C2F76BC032F00A95BB0CDD1CEE1CFF1CB6
:10705000F9CF01D0D5CFB7FE089590E8B91611F455
:10706000D0FE08959FEFD91AE90AF90A09F40395A9
:107070000895DD92ED92FD920C930895502F2D2DE1
:107080003E2D4F2D612F08952DEC3CEC4CEC5DE333
:1070900066270FC099DFF2DFDD24EE2490E8F92E99
:1070A0000FE307C096DF05C02227332740E251E4F3
:1070B0006627552351F1002381F190DF71F11627E6
:1070C000005850580894050B18F407FD03C025C05C
:1070D00007FD23C0469537952795F694E794D794F6
:1070E00022D0FF202AF0DD0CEE1CFF1C015073F0B3
:1070F0009D2D969548F0DD203AF4EE202AF491E09B
:10710000D90E9927E91EF91E7BCF07C09FE7092FEB
:10711000F92A9FEFD92EE92E0895DD24EE24FF24CD
:107120000027112708959F929924AA24BB2488E15F
:10713000D216E306F40628F0D21AE30AF40A0894F9
:1071400001C08894991CAA1CBB1CDD0CEE1CFF1C02
:107150008A9571F7D92CEA2CFB2C9F9008953EDF7D
:10716000E1F25038D1F21627005850580894051F04
:1071700012F418F4CBCF08F0D0CF0AD0FF202AF0B9
:10718000BB0CDD1CEE1CFF1C3BCF0F5FFBF138CFAF
:107190009F929924AA24BB24992788E1990CAA1CC0
:1071A000BB1CDD1CEE1CFF1C30F4920EA31EB41E93
:1071B000D91EE91EF91E8A9589F79F90089509DF67
:1071C0000DDF503829F090E869270CC00AF045D04F
:1071D00017CF5FE322273327442701C0FADEFEDE04
:1071E0005038B1F3003899F3902F951B8BF312F4BC
:1071F00034D0FACF983118F022273327442798301B
:1072000028F0232F342F44279850F9CF992329F0C1
:107210004695379527959A95D9F7912F962742F05D
:1072200014D0B0F6F794E794D7940F5F8BF66ECF37
:1072300010D051F008F4BEDEFF2052F2DD0CEE1C3F
:10724000FF1C0150CBF762CF68CFD20EE31EF41EB5
:107250000895D21AE30AF40A0895DF92EF92FF929A
:107260000F931F93D22EE32EF42E052F162F6F911E
:107270005F914F913F912F910895C89531960020CD
:107280000895FBDFD02CF9DFE02CF7DFF02CF5DFE1
:10729000002D0895F2DF202DF0DF302DEEDF402DA0
:1072A000ECDF502D089507FB00680EF40F7757FBB5
:1072B00050680EF45F7707FD02C057FF05C0D21675
:1072C000E306F406050708952D153E054F05500702
:1072D000089500240D280E280F28002A0020089564
:1072E00091E005C092E003C094E001C098E0C5DFE2
:1072F0000D929A95E1F70895E80FF91FF1CF880FE5
:10730000991F880F991FE80FF91FEECF882311F4FA
:10731000992329F00E943D39E9F70197D9F708959B
:1073200091E0882321F08894991F8A95E9F7892FA5
:10733000909508952E2E3F2E992781918D3209F038
:1073400093958823D1F79A95E22DF32D112361F0BF
:10735000091718F011F0101B01C0191B28F021F0BB
:1073600080E28D931A95E9F780818D3219F48D931F
:10737000319604C0222311F08BE28D93091738F067
:1073800031F0091B21F080E38D930A95E9F7819193
:107390008D938823E1F7332351F0EA2FFB2F3196A9
:1073A00033958E9182933A95E1F78EE28C9308950E
:1073B00099278D9193958823E1F7939511968C9356
:1073C00011978E919A95D1F70895EA2FFB2F0024FB
:1073D0004C918D9103948E32E1F711248D91139489
:1073E0008823E1F71A94101640F41197202F2119E1
:1073F000239580E38D932A95E9F7113039F5992784
:10740000AE2FBF2FA00DB91FA00FB91F8C919C9359
:10741000853308F421C031E08E918E32E9F38D324C
:1074200041F0830F8A3319F480E331E001C0332740
:107430008C93AE1789F7332341F0AE2FBF2FB8DFFF
:1074400081E34D3209F43196808308958827E00D59
:10745000F81FE00FF81F80830895040F151F261FE3
:10746000371F0895041B150B260B370B08950417BF
:107470001507260737070895000F111F221F331F16
:10748000089500951095209530950F5F1F4F2F4F51
:107490003F4F0895019110810EC0019111912191EA
:1074A00030810BC00191108117FF05C03FEF2FEF16
:1074B00004C0008111272227332737FF03C0E1DFF3
:1074C0008DE28D93CF93DF93CF92DF92EF92AA2438
:1074D000BB24CC24DD24EE2440E2CAE0DD2755E0C5
:1074E00093E38881890F87FD9F7083FD907F891BBF
:1074F00089935A95A9F7C0DFAA1CBB1CCC1CDD1CC4
:10750000EE1C4A9551F7E894EFE0FF2782910ED0E8
:10751000EB30E0F71EF068948A2D0CD088278D930D
:10752000EF90DF90CF90DF91CF910895982F8295C3
:1075300001D0892F8F70805D26F0803309F4089583
:1075400068948D93089500271127222733271DD093
:107550008A3328F4803318F005D015D0F9CF0EF413
:1075600090CF089580538F93402F512F622F732F08
:1075700083DF82DF72DF80DF8F919927080F191F69
:10758000291F391F08958D910895E894FCDF8032FA
:10759000E9F38B32D9F38930C9F38D3211F4689451
:1075A000F2CF089588278D93089581918D93882334
:1075B000E1F7089594E081918D939A95E1F708950C
:1075C00009919191992351F08A95D9F73197819139
:1075D0008D930A9519F08823D1F70895E3CFE199A7
:1075E000FECFEEBBFFBB3196089591E001C092E063
:1075F000F6DFE09A8DB38D939A95D1F70895FF93B6
:107600005527F8E0469508F4500F57954795FA9599
:10761000D1F7FF910895FF93881BF9E0001FFA95B9
:1076200011F4FF910895881F841B18F4840F889427
:10763000F5CF0894F3CF8FEF83959D919923E1F7D0
:107640000895E89463F80895689463F80895BCDC9D
:107650000F770895B9DCC2DC0395AAF087E1DD0C51
:10766000EE1CFF1C8A9589F00A95CAF7FF205AF094
:1076700000240D280E280F28002039F00A95DD0C73
:10768000EE1CFF1CDAF70A95BBCC47CD9DDC85E0EC
:1076900041D10F7723E839EF42E25EE360DDDBDFC3
:1076A000E8DC139727D08A3F40F000688D3F18F43C
:1076B00090DD80E803C057D192DD88278483DEDC2B
:1076C0004EDDD7DC139729EA3EE64CE952EC47DD64
:1076D00022E332E541E852E40AD122ED32EE4DE9EF
:1076E00051EC05D120E93FEF4FE75FE378DD84817E
:1076F00008271DC1802F9F2D991F881F991F881F44
:1077000008950BCD61DC0023E2F3E3DD19F4FEDC28
:107710000068089585E0FED0FF0C001F04830FE78A
:107720000695F79420D150685ADDA3DC139721E425
:1077300038E743ED5BEB13DD27E831ED43E15DE333
:10774000D6D02EE03CE343EC5DEBD1D022E83DEA1D
:107750004BE25EE3CCD02CEE32E846E75EEBC7D0DE
:1077600020E931EE49EA5EE3C2D020E83FEE4FEF78
:107770005EEBBDD024EC3FEF4FE75FE3B8D079DCA0
:10778000139784818F5799F02AF4D82E0FEFE02EAB
:10779000F02E04C0D82EEE24FF24002739DC28E187
:1077A00032E741E35FE3DBDC14DC349718DDBFC074
:1077B0000BDC80E003C008DC802F8078882321F078
:1077C000DF92EF92FF920F938F9308DC802F8395C7
:1077D00012F4A3DC1BC080958A95885E0AF415C05C
:1077E00088501AF40CD0D92210C0DD2488501AF425
:1077F00006D0E9220AC0EE2402D0F92206C09FEF8B
:107800008770990F8A95EAF70895FADB8F9188239C
:10781000D9F35F914F913F912F910F9344DD0F91D9
:1078200099F390F3A0D05068DACC70DC80C0CCDB48
:1078300086E070D005830F772BE33AEA48EB5FE3ED
:107840008EDC17DC139741D028F4858188236AF7F2
:1078500064DC6DC08F778483B7DB3497FCDE09DC92
:10786000139723E632E446E357EB79DC29ED37EA58
:107870004AE159E33CD026E538E14EEA5AEB37D0ED
:1078800026E53CE84DE15CE332D02DEC37E543E6FC
:107890005DEB2DD02DEE3DEF45E75EE328D028E1EE
:1078A00032E741E35FEB23D05ED099DCE7DBDD24F8
:1078B000EE24FF2404818FE7080F0695F794F9DB87
:1078C0008581881F08F4E7DB32C088DB88270395B1
:1078D00012F48894089507301AF0812F08940895BF
:1078E000FF1C881F0A95E2F7812B8894089577DCA6
:1078F00070DB349734CC68DB0F93AF93BF930F7773
:1079000002DFFF91EF9165DB2ADC92DF8F918078B7
:10791000082B08950FB6F8944A925A92E42DF52D4B
:10792000A42DB52D480E8827581E0FBE08950FB6FA
:10793000F894599049900FBE089546DB002331F02A
:107940002BED3FE049EC5FEB4ADCA1CEE6CB3CDB24
:10795000802FFF0C001F901728F4091B881F079524
:10796000F7940895DACB5FE340E8332722270895A0
:107970002BDB0F930F772DDC1FDF8F918078082B87
:107980000895CBCB21DB0023E2F3D9F388E0C2DFFB
:1079900070DB1196FF0C001F8FE7080F0795F79417
:1079A0000695F79483E08F9369DB63DB13970CDB19
:1079B00080DB0FDB389713DC91E0CADF8F918A956B
:1079C00011F08F93F1CFB3CFC3F5283F0000E4420D
:1079D000000000400000444200009643000048427E
:1079E000000070C2000034430AD71F41000020C1CC
:1079F00000007A440000C8420000204100C07944E1
:107A0000180D8F4D0000FA44003C1C46103C703DA0
:107A10000000F041713D1A4100008041000080BF2C
:107A20000000A0410000803F0B2D343EE12E654256
:107A30000AD7233CCDCCCC3D3F2F5E76202E2D4067
:107A400025263031323334353637383941424344D4
:107A500045464748494A4B4C4D4E4F50515253545E
:107A600055565758595A0000202020202020202009
:107A700020202020202020202020200053575200AA
:107A80005A00524C000050485300525800005853BE
:107A90000000202020205E20200020200000200068
:107AA0004D00434C205E2020200051004257205EB4
:107AB00020202000420047454E455254000020201F
:107AC0004D4F444500004820000033003200312073
:107AD0000000260025004000203000002035000076
:107AE0003130000031350000323000003235000006
:107AF00033300000303000003430000035300000FA
:107B0000363000002033000020360000203900000D
:107B10003132000031380000564E4100494D5000CE
:107B2000574F4200504841005300460043004C006C
:107B30005200495733484556202F20504133434B7C
:107B40005200414E54454E4E4120414E414C5953F6
:107B50004552000056302E37204D415834205350A6
:107B60003353574A000055534200464F5220555355
:107B700042204D4F44450000505245535320465536
:107B80004E4354494F4E204B455900004445464111
:107B9000554C54204C4344204D4F44450000560062
:0C7BA000490057005000540076005E00C1
:00000001FF
